:0200000480007A
:10000000B72F0000938F0F8073900F3015A8130047
:100010000000130000001300000013000000130094
:100020000000130000001300000013000000130084
:100030000000130000001300000013000000010086
:10004000970200009382020C73905230814001416C
:100050008141014281420143814301448144014580
:100060008145014681460147814701488148014950
:100070008149014A814A014B814B014C814C014D20
:10008000814D014E814E014F814F971102009381A6
:1000900021D3170502001305E556979503009385B4
:1000A000257E01461122170502001305E548970534
:1000B00002009385A5500146C52817A50300130526
:1000C000657C97B503009385A57B37B6ABAB13066C
:1000D000B6BAD92817B103001301C17AEF60E075F1
:1000E000860293D21200F512638802008242110147
:1000F0006F00001073002030824211017300203025
:10010000711116C0F3222034E3CC02FC82421101AB
:10011000130141F806C20AC40EC612C816CA1ACC88
:100120001ECE22D026D22AD42ED632D836DA3ADCC7
:100130003EDEC2C0C6C2CAC4CEC6D2C8D6CADACC97
:10014000DECEE2D0E6D2EAD4EED6F2D8F6DAFADCA7
:10015000FEDE73252034F32510340A8601A07310C7
:10016000153492402241B2414242D2426243F243AC
:10017000025492542255B2554256D2566257F25703
:10018000064896482649B649464AD64A664BF64B33
:10019000065C965C265DB65D465ED65E665FF65F83
:1001A0001301C1077300203010C16374B50011053D
:1001B000E5BF828000000000000000000000000099
:1001C000000000000000000000000000000000002F
:1001D000000000000000000000000000000000001F
:1001E000000000000000000000000000000000000F
:1001F000197106C00AC20EC412C616C81ACA1ECC8D
:1002000022CE26D02AD22ED432D636D83ADA3EDCC6
:1002100042DEC6C0CAC2CEC4D2C6D6C8DACADECC96
:10022000E2CEE6D0EAD2EED4F2D6F6D8FADAFEDCA6
:100230009702020083A2823323A02200F32210340B
:1002400096DEEF00002B170102000321213202414C
:10025000F65273901234B72200009382028873A082
:10026000023082403242C2425243E24372448254DC
:100270001255A2553256C2565257E2577258864806
:100280001649A649364AC64A564BE64B764C865C1A
:10029000165DA65D365EC65E565FE65F0961730059
:1002A0002030970202009382E23523A0120023A29D
:1002B000220023A4320023A6420023A8520023AA2E
:1002C000620023AC720023AE820023A0920223A21C
:1002D000A20223A4B20223A6C20223A8D20223AA06
:1002E000E20223ACF20223AE020323A0120523A2F2
:1002F000220523A4320523A6420523A8520523AADA
:10030000620523AC720523AE820523A0920723A2C7
:10031000A20723A4B20723A6C20723A8D20723AAB1
:10032000E20723ACF207EF40104D17010200032152
:10033000E1230241F65273901234B72200009382F7
:10034000028873A0023082403242C2425243E243EA
:10035000724482541255A2553256C2565257E25731
:10036000725886481649A649364AC64A564BE64B45
:10037000764C865C165DA65D365EC65E565FE65FB1
:10038000096173002030970202009382A22783A0A4
:10039000020003A1420083A1820003A2C20083A243
:1003A000020103A3420183A3820103A4C20183A427
:1003B000020203A5420283A5820203A6C20283A60B
:1003C000020303A7420383A7820303A8C20383A8EF
:1003D000020403A9420483A9820403AAC20483AAD3
:1003E000020503AB420583AB820503ACC20583ACB7
:1003F000020603AD420683AD820603AEC20683AE9B
:10040000020703AFC20983AF820782807370043092
:10041000197106C00AC20EC412C616C81ACA1ECC6A
:1004200022CE26D02AD22ED432D636D83ADA3EDCA4
:1004300042DEC6C0CAC2CEC4D2C6D6C8DACADECC74
:10044000E2CEE6D0EAD2EED4F2D6F6D8FADAFEDC84
:100450009702020083A2821123A0220086DEEF20F1
:10046000405417010200032161100241F6527390BB
:100470001234B72200009382028873A002308240B7
:100480003242C2425243E243724482541255A25550
:100490003256C2565257E257725886481649A649F4
:1004A000364AC64A564BE64B764C865C165DA65DD0
:1004B000365EC65E565FE65F09617300203073707A
:1004C000043001A07310453082807325403073F0F2
:1004D00043308280970700009387A7FE232EB5FE46
:1004E0002322C5FA232635F82320F5F8130505F84D
:1004F0008280411106C6EF40702DEF10703001E58B
:10050000B24041018280B24041016F20804993078F
:1005100085007D575CC118C55CC51CC9232005003A
:1005200082802328050082805C41DCC1984798C501
:1005300098474CC38CC788C91C4185071CC1828061
:100540009041FD57130785006314F60039A83E87D4
:100550005C439443E37DD6FEDCC18CC798C54CC395
:1005600088C91C4185071CC1828018495C43EDB7CE
:10057000584114451C4914C71845544154C3D84325
:100580006314A7001845D8C32328050088437D15A8
:1005900088C382803041AE8701CE4C455841B29528
:1005A0004CC563E4E5000C414CC53E856F30904678
:1005B0008280411122C406C62A8426C2EF20103848
:1005C0003C44635BF0025C5085CB9304440209A871
:1005D0003C44FD173CC43C446350F0025C5089CF5E
:1005E0002685EF20207E6DD5EF20101E3C44FD17A0
:1005F0003CC43C44E344F0FEFD573CC4EF2050367D
:10060000EF20D0337C40635BF0021C4885CB930421
:10061000040109A87C40FD177CC07C406350F002B7
:100620001C4889CF2685EF20E0796DD5EF20D019C1
:100630007C40FD177CC07C40E344F0FEFD577CC04D
:100640002244B240924441016F20903129CD0111E2
:1006500022CC2A8406CE26CA4AC84EC62E89EF204E
:10066000F02D24404C5C832904002685EF50907EB9
:100670007D57232C0402B3079540CE974E9578C042
:1006800048C0232434015CC438C4631109021C48E7
:100690008DE7EF20F02CF2406244D2444249B24947
:1006A0000545056182807370043001A013050401C3
:1006B000B93D13054402A13DE9BF13050401EF2034
:1006C00060708547E317F5FC9133E1B701E573707E
:1006D000043001A0011126CA4AC84EC606CE22CC5B
:1006E000AA842E89B289A5C9EF50D0761305550585
:1006F000EF30101A2A8435C5930745051CC144DC28
:1007000023202405EF20902324404C5C032904007F
:100710002685EF503074FD56232C0402B307954014
:100720003307A900CA9774C058C05CC434C4130509
:10073000040123242401E13B13054402C93BEF20BB
:100740003022230834052285F2406244D2444249D3
:10075000B2490561828013054005EF3070132A8489
:1007600001E57370043001A000C051BF01E5737052
:10077000043001A06375B5007370043001A041110D
:1007800022C409462E84814506C6893711C500DD7D
:10079000B2402244410182807370043001A05D7137
:1007A00086C6A2C4A6C2CAC04EDE52DC56DA5AD8E9
:1007B0005ED632C6630A051C6382051C89476399AD
:1007C000F600585D85476305F7007370043001A09B
:1007D0003689AE842A84EF20B00111E5B24781C783
:1007E0007370043001A0EF207015185C5C5C014B45
:1007F000894BFD59130A0401930A44026365F70CFF
:1008000063077919B2476381072463150B00280831
:10081000EF20606EEF20D014EF104075EF20101223
:100820007C4063943701232204043C4463943701E1
:1008300023240404EF20D0126C002808EF20C06DA0
:10084000631E051EEF20900F185C5C5C630CF70ABA
:10085000EF201011EF20900E3C44634FF00039A8B8
:100860005685EF20205619C1EF2000763C44FD1735
:100870003CC43C446354F0005C50FDF32324340535
:10088000EF20100EEF20900B7C40634FF00039A852
:100890005285EF20205319C1EF2000737C40FD17D3
:1008A0007CC07C406354F0001C48FDF323223405D7
:1008B000EF20100BEF109010054BEF203008185C64
:1008C0005C5CE37FF7F230406305060C631F09129E
:1008D0000844A685EF3010141C4434405840B697A5
:1008E0001CC463EAE70A1C5C14405850850714C412
:1008F0001CDC5DC713054402EF20C04C8547631123
:10090000F50AC9A8EF20D005B2455285EF20402D49
:10091000EF20D0023C44634FF00039A85685EF2009
:10092000604A19C1EF20406A3C44FD173CC43C4476
:100930006354F0005C50FDF323243405EF20500293
:10094000EF20C07F7C40634FF00039A85285EF2034
:10095000604719C1EF2040677C40FD177CC07C4098
:100960006354F0001C48FDF323223405EF20407F40
:10097000EF10D00431F1593C054B81B73C41E38F76
:1009800007E27370043001A07370043001A030409E
:1009900021E61C4085C71C5C585085071CDC39FBD0
:1009A000EF20007C0545B640264496440649F2599E
:1009B000625AD25A425BB25B616182804840EF204A
:1009C000406F1C5C58502322040085071CDCE31395
:1009D00007F279D5253CE9B74844A685EF30900366
:1009E0003C4058441440B307F0403E9758C4637CE1
:1009F000D7025840BA975CC409475C506306E902C5
:100A0000185C050718DCC9DFF5B54844A685EF304A
:100A100070003C4058441440B307F0403E9758C41F
:100A2000E37CD7FCF9B75C50185C79DB185C7D1768
:100A300018DC185C050718DCA5D76DBD2285953E2E
:100A4000EF10C077014585B7EF2080710145A1BF48
:100A5000411126C2AA841305400522C406C6EF3000
:100A600020632A8415CD232C0502FD577CC1054740
:100A7000410558DC3CC42322040023200400232425
:100A80000400232604002320040423089404413492
:100A900013054402AD3C8146014681452285013360
:100AA0002285B24022449244410182800DC5411109
:100AB00022C426C206C64AC0032945002A84EF2064
:100AC00060528144630CA900B24022442685024949
:100AD0009244410182807370043001A05C448544DB
:100AE000FD175CC4F5F381460146814522854539F1
:100AF000E1BF397106DE22DC26DA4AD84ED652D45E
:100B000032C635CD8149DDC13689AE842A84130AC7
:100B100005012DA0EF20C064EF2040626C00280882
:100B2000EF20803F31E1EF206061185C5C5C630581
:100B3000F702EF20E062EF20A0628549EF2000601D
:100B4000185C5C5C6360F704B24799CFE39409FCDE
:100B50002808EF20403A7DBFEF208060B2455285E3
:100B6000EF2000086530C1BFEF20805FF250625473
:100B7000D2544259B259225A014521618280737080
:100B8000043001A0304015EE1C4095C71C5C585045
:100B900085071CDC39E7EF20A05CF2506254D25488
:100BA0004259B259225A0545216182803C41A9DF50
:100BB0007370043001A04840EF20A04F23220400AE
:100BC000F1B7631909020844A685EF30A0641C44FC
:100BD00034405840B6971CC4E3EAE7FA1C401CC4F2
:100BE00075B713054402EF20E01D8547E315F5FABC
:100BF000313855B74844A685EF30C0613C40584471
:100C00001440B307F0403E9758C46375D70058406E
:100C1000BA975CC48947E31BF9F61C5CA5DB1C5C36
:100C2000FD171CDCA5B7397106DE22DC26DA4AD8AE
:100C30004ED652D432C66301050E81446388050C3A
:100C4000B6892E892A84130A450231A0EF2040512B
:100C5000EF2000518544EF20604E1C5CBDE3B2479D
:100C600095CF8DC8EF20C04FEF20404D6C00280875
:100C7000EF20802A05E5EF20604C1C5CE1FBEF20B3
:100C8000204E1C409DC7B2455285EF107075EFF0A5
:100C9000EFF77DBF2808EF200026E9B7EF20404C92
:100CA000F2506254D2544259B259225A014521613C
:100CB0008280EF20A0484840EF208035EF20404A56
:100CC000D9B73040444409CE5840B387C4005CC40F
:100CD00063E4E7001C405CC44C444A85EF30805319
:100CE000639F09021C5C1840FD171CDC01E7EF2024
:100CF000A04B48C01C489DC713050401EF20800C81
:100D000085476311F502EFF06FF029A83C41E389B4
:100D100007F27370043001A07370043001A05C50BE
:100D200044C481EFEF20C043F2506254D254425980
:100D3000B259225A05452161828013054402EF20F1
:100D400060086DD1C9B725C1B1C9011122CC26CA2D
:100D50004AC852C406CE4EC68947B68432892E8A06
:100D60002A846399F600585D85476301F70673701E
:100D7000043001A0EFF06FF5185C5C5CAA89636732
:100D8000F70281444E85EFF0EFF3F240624426858E
:100D90004249D244B249224A056182803C41D5D7BA
:100DA0007370043001A07370043001A0304049E238
:100DB0001C40DDCB1C5C7D5785071CDC3C446388F4
:100DC000E7083C44854485073CC46DBFEFF0EFEF76
:100DD000185C5C5CAA89636DF702304071DA4844A4
:100DE000D285EF3020433C4058441440B307F040D4
:100DF0003E9758C46375D7005840BA975CC489477A
:100E0000E39AF4FA1C5CDDD71C5CFD171CDC5DB7B3
:100E1000304059DE4844D285EF30C03F3C40584412
:100E20001440B307F0403E9758C4E367D7FCD9BFDE
:100E3000DDF40844D285EF30E03D1C443440584096
:100E4000B6971CC4E3E8E7F61C401CC4A5B75C5089
:100E500085448DDB13054402EF10D07605D5E303FE
:100E600009F22320990039BF4840EF208024232233
:100E7000040089B731CD3C4181C77370043001A0B3
:100E80001C41B1CB011122CC26CA2A844AC84EC6C5
:100E900006CE2E89EFF06FE3185C5C5CAA89814472
:100EA000637DF7001C5C7D5785071CDC3C4463892F
:100EB000E7023C44854485073CC44E85EFF08FE053
:100EC000F240624426854249D244B249056182809B
:100ED0007370043001A05C41D5D77370043001A059
:100EE0005C5099E38544D1BF13054402EF10906D27
:100EF00075D9E30909FE85472320F900E5B7397163
:100F000006DE22DC26DA4AD84ED652D456D232C673
:100F10006302051C638A051AB68AAE892A84EF200B
:100F2000200D11E5B24781C77370043001A0EF2096
:100F3000E0201C5C63920714B247638E070A2808FE
:100F4000EF10707BFD5413094402130A0401EF20D3
:100F50002021EF10A001EF20601E7C4063949700D9
:100F6000232204043C446394970023240404EF20C8
:100F7000201F6C002808EF10307A63130518EF204B
:100F8000E01B1C5CADCFEF20A01DEF20201B3C44DC
:100F9000634FF00039A84A85EF10D06219C1EF20E5
:100FA000A0023C44FD173CC43C446354F0005C5038
:100FB000FDF324C4EF20C01AEF2040187C40634F9B
:100FC000F00039A85285EF10F05F19C1EF10D07F03
:100FD0007C40FD177CC07C406354F0001C48FDF34E
:100FE00064C0EF20E017EF10601DEF2020151C5C9F
:100FF000C1E7B247A9FFEF20A016014555A0EF2099
:1010000020161C40DDC7B2454A85EF10703DEF2029
:10101000E0123C44634FF00039A84A85EF10905A23
:1010200019C1EF10707A3C44FD173CC43C44635432
:10103000F0005C50FDF324C4EF208012EF2000107C
:101040007C40634FF00039A85285EF10B05719C1AA
:10105000EF1090777C40FD177CC07C406354F0001B
:101060001C48FDF364C0EF20A00FEF10201531C91C
:10107000EF20C00C1C5CB5DFCE8522854444EFF028
:101080006FD1639C0A041C5C1840FD171CDC01E74F
:10109000EF20801148C01C48A1EFEF20600C0545EF
:1010A000F2506254D2544259B259225A925A216192
:1010B0008280EF20A0084840EF109075EF20400A92
:1010C00099B7EFF0AFB46DB73C41E38707E47370B5
:1010D000043001A07370043001A05C5044C4D5DF1B
:1010E00013054402EF10104E4DD9EFF02FB275B733
:1010F00013050401EF10104D8547E310F5FAF5B71D
:101100002285EFF00FCBEF10600B014551BF1DC9D9
:10111000411122C44AC006C626C244412E892A84EF
:10112000EF10506C6383A40281464A868145228574
:10113000F93385476300F502B240224492440249E4
:10114000410182807370043001A05C44054585072D
:101150005CC4DDB75C4485075CC4F9BF15CDADC97F
:10116000011122CC26CA4AC84EC652C42A8406CED1
:101170003289AE89EFF06FB51C5C2A8A814485E321
:101180005285EFF02FB4F240624426854249D244A2
:10119000B249224A056182807370043001A0304058
:1011A00001CE4C445C40B2954CC463E4F5000C4065
:1011B0004CC44E85EF3000061C5C7D57FD171CDCCF
:1011C0007C40638CE7007C40854485077CC04DBF34
:1011D0003C41D9D77370043001A01C4899E3854481
:1011E00045B713050401EF10F03D75D9E30909FE79
:1011F00085472320F900E5B721C93C41A1CDA1CB0A
:10120000011122CC26CA4AC852C42A8406CE4EC630
:101210002E8AEFF08FAB1C5C2A89814491CB832905
:10122000C400D2852285EFF0EFB685442326340131
:101230004A85EFF02FA9F240624426854249D24404
:10124000B249224A056182807370043001A0737034
:10125000043001A0EDDF7370043001A001E573706C
:10126000043001A0411122C42A8406C6EF10106D7B
:10127000005CEF10F06EB240228522444101828072
:1012800001E57370043001A0411106C622C42A840E
:10129000EF10D06A1C5C405C1D8CEF10706C2285D6
:1012A000B24022444101828019C1085D828073707E
:1012B000043001A01DCD978703009387A758D8431A
:1012C000630CE502D847630CE504D84B6307E504DB
:1012D000D84F6302E504D853630DE502D85763087D
:1012E000E502D85B6303E502D85F630EE5006F207B
:1012F000506C7370043001A001470E07BA9723A009
:1013000007006F20106B1D47CDBF1947FDB715476C
:10131000EDB71147DDB70D47CDB70947F9BF054711
:10132000E9BF684582806CC58280034505058280DF
:1013300009C5085D1335150082807370043001A063
:1013400019C51C5D485D1D8D1335150082807370B5
:10135000043001A0978703009387C74E984305C3C5
:10136000984705C7984B05C7984F05C7985305C7B9
:10137000985705C7985B15C7985F15C382800147CA
:101380000E07BA978CC3C8C382800547D5BF0947EB
:10139000C5BF0D47F5B71147E5B71547D5B71D4789
:1013A000C5B71947F1BF978703009387A749D8436B
:1013B0006308E502D847630BE502D84B630AE502F0
:1013C000D84F6309E502D8536308E502D85763078D
:1013D000E502D85B6308E502D85F6303A702828059
:1013E00001470E07BA9723A0070082800547D5BFA3
:1013F0000947C5BF0D47F5B71147E5B71547D5B73D
:101400001D47C5B71947F1BF411122C426C24AC0C2
:101410002A8406C6AE843289EF1050527840FD57B8
:101420006314F700232204043844FD576314F700C3
:1014300023240404EF10D0521C5C99E74A86A68549
:1014400013054402EF10D00CEF10504F3C44635B87
:10145000F0025C5085CB9304440209A83C44FD177C
:101460003CC43C446350F0025C5089CF2685EF10A9
:1014700070156DD5EF1050353C44FD173CC43C440D
:10148000E344F0FEFD573CC4EF10904DEF10104BBD
:101490007C40635BF0021C4885CB9304040109A8DF
:1014A0007C40FD177CC07C406350F0021C4889CF13
:1014B0002685EF1030116DD5EF1010317C40FD17EF
:1014C0007CC07C40E344F0FEFD577CC02244B24027
:1014D0009244024941016F10B0481DC179714ECE4E
:1014E00052CC06D63E8A22D426D24AD056CA5AC8F0
:1014F0005EC6A547BA8963F8E7007370043001A09F
:101500007370043001A02A8BAE843289B68BC28AF4
:101510006307082213050006EF2090372A84630B27
:1015200005200A09232855034A869305500A568543
:10153000EF20505C03C704001C587119230AE40211
:1015400003C704003E991379C9FF79C783C7140004
:10155000A30AF40283C71400E1C383C72400230B4A
:10156000F40283C72400CDCB83C73400A30BF4025D
:1015700083C73400D5C383C74400230CF40283C758
:101580004400D9CB83C75400A30CF40283C7540092
:10159000C1C783C76400230DF40283C76400ADCFC5
:1015A00083C77400A30DF40283C77400B5C783C753
:1015B0008400230EF40283C78400B9CF83C794004C
:1015C000A30EF40283C79400A1CB83C7A400230F0A
:1015D000F40283C7A400A9C383C7B400A30FF40215
:1015E00083C7B40095CB83C7C4002300F40483C72A
:1015F000C4009DC383C7D400A300F40483C7D400F0
:1016000081CF83C7E4002301F40483C7E40089C7C2
:1016100083C7F400A301F404930A44005685A30190
:1016200004042326340323283405232A0404EFE08A
:101630005FEF13058401EFE0DFEEA947B387374181
:10164000232C040400C81CCC40D023220404232EE5
:1016500004045E86DA854A85EFE0DFE708C06304AC
:101660000A0023208A007370043017F9010013095F
:1016700029EE8327090097F40100938424EF91C792
:1016800098409C407C4385077CC317F701001307F3
:10169000E7EC1C43850797F6010023A1F6EC9C407C
:1016A000C5CB8327090017FB0100130B6BFD89EBEA
:1016B0009C40DC5763E6F90097F7010023A887EA0E
:1016C00097F701009387C7E79C4317F701001307BB
:1016D00067E848541843850797F6010023A2F6E609
:1016E0003CC46376A70097F7010023A5A7E6D14580
:1016F000EF405076D6855A95EFE01FE38327090027
:1017000081C79C40FC43B5E383270900054499C782
:101710009C40DC5763F43701EFE05FCF2285B25085
:10172000225492540259F249624AD24A424BB24B75
:10173000456182805685EF20D0277D54C5B71315AB
:101740002600EF20F014AA8AE31605DC7D54F9B7D1
:1017500097F7010023AC87E0184385476301F70240
:1017600017FB0100130BCBF1A1BF984094407C43C1
:10177000FD177CC3FC42C9FB7360043071B7014A9A
:1017800017FB0100130BCBEFA94B5285D145EF405E
:10179000706C050A5A95EFE09FD7E3187AFF97FB24
:1017A0000100938B6BFA5E85EFE07FD617FA01009C
:1017B000130ACAFA5285EFE09FD517F50100130509
:1017C00025FBEFE0DFD417F501001305A5FBEFE0E3
:1017D0001FD417F50100130525FCEFE05FD397F741
:1017E000010023A377D997F7010023AD47D7C9BDDF
:1017F000411122C406C626C24AC02A84737004302E
:1018000097F401009384C4D49C40F9E311E497F762
:1018100001009387A7D58043130944004A85EFE070
:101820003FD51C5489C713058401EFE07FD4CA85D6
:1018300017F50100130505F5EFE01FCF97F701003D
:10184000938707D2984397F70100938767CF9C430C
:10185000050797F6010023A5E6D09840850797F67F
:10186000010023AFF6CC01CB97F70100938707D097
:101870009843784349EF9C40B1C797F7010093879D
:10188000E7CE9843630F870873700430984039EBB4
:1018900017F70100130747CD14439442A5E27D5783
:1018A00097F6010023ACE6C8984009CF98437843E7
:1018B00011CB984394437C43FD177CC3FC4299E3CE
:1018C00073600430B2402244924402494101828054
:1018D00097F70100938787C998439C437C4385070A
:1018E0007CC32DB794439843F8420507F8C217F715
:1018F0000100130767C714439442D5D218435847D1
:101900005847584397F6010023AAE6C271BF98438F
:1019100094437C43FD177CC3FC42B1FF73600430E9
:1019200099BF97F70100938727C19C4381C77370C4
:10193000043001A02244B2409244024941016FE0C8
:10194000FFAC41C517F70100130747C21443814795
:10195000638BA606411106C622C426C273700430EA
:1019600097F601009386C6BE9C4291C710431C4364
:101970007C4285077CC29C42AA84404981C71C43A3
:10198000FC43B9E797F70100938707BE9C43638B3D
:10199000870497F701009387E7BC9C43638487041F
:1019A00097F70100938747DF6309F40297F7010077
:1019B000938747DD6301F4028547B2402244924495
:1019C0003E85410182803E8582807370043001A093
:1019D000EF40105C45BF9147CDB79C5493B71700BB
:1019E0008907E1BF8947D1BF7370043097F70100C1
:1019F000938707B6984309EF15C59C43485581CB9B
:101A000097F70100938787B69843784315E3828060
:101A100017F70100130787B514431843F842050769
:101A2000F8C261FD17F70100130747B40843F1B787
:101A3000984394437C43FD177CC3FC42E9FB7360ED
:101A400004308280411122C42A8406C6EFE0FFA739
:101A500011E497F70100938767B180434054EFE0AA
:101A60007FA6B2402285224441018280A54763F5CA
:101A7000B7007370043001A0011122CC06CE26CA33
:101A80004AC84EC652C42A847370043017F9010044
:101A9000130909AC83270900CDEF71C43C48638862
:101AA000F50817F70100130767AC63FCB700144390
:101AB000638C860C18434457B3B4950093C4140048
:101AC00029A00443818C93B4140058546383E70A1B
:101AD0001C4C2CC863C60700A947B385B7400CCC83
:101AE00093172700BA97584897F90100938949B985
:101AF0008A07CE97631AF702130A44005285EFE073
:101B00003FA797F701009387E7A448549C4363F6E7
:101B1000A70097F7010023AFA7A2D145EF4090336C
:101B2000D2854E95EFE05FA099C0EFE03F8E83270E
:101B3000090081CB97F70100938747A39C43FC439F
:101B40009DEBF2406244D2444249B249224A0561C7
:101B5000828097F70100938767A198439C437C4359
:101B600085077CC305FC97F70100938727A0804376
:101B700035B74CD4B1BF6244F240D2444249B24975
:101B8000224A05616F40D040814481B725C10111CF
:101B900026CA97F401009384649D9C4006CE22CC13
:101BA0004AC84EC6638DA7027370043017F901004E
:101BB0001309099A8327090091C798409C407C43E8
:101BC00085077CC3584997F701009387E7BC6302F8
:101BD000F7028327090081C79C40FC43A5EBF24034
:101BE0006244D2444249B249056182807370043034
:101BF00001A01C5517F70100130787B7E38BE7FC1B
:101C0000E9FB930945002A844E85EFE07F9697F71C
:101C100001009387279448549C4363F6A70097F7E5
:101C2000010023A9A792D145EF40D02297F70100E8
:101C3000938707A53E95CE85EFE01F8F9C405854B3
:101C4000DC57E368F7F8EFE06FFC61B76244F240FD
:101C5000D2444249B24905616F40903315CD01111C
:101C600022CC26CA4EC62A8406CE4AC8EFE0FF859B
:101C7000584897F70100938727B2AA8981446300E7
:101C8000F7024E85EFE01F84F24062442685424908
:101C9000D244B249056182807370043001A01C54A3
:101CA00017F501001305C5ACE38DA7FCF9FB97F709
:101CB0000100938767889C43A9EB97F701009387FE
:101CC000E78A9C43445413094400DC574A85B3B463
:101CD000F400EFE0FF8997F701009387A787485446
:101CE0009C4393C4140063F6A70097F7010023A355
:101CF000A786D145EF40101697F7010093874798C4
:101D0000CA853E95EFE05F82ADBF93058401EFE0A9
:101D1000BF8185BF0111056506CE22CC26CA4AC8FF
:101D20004EC652C456C25AC0EF208036630E051A02
:101D3000AA8413050006EF20A0352A84630A051C37
:101D400005669305500A04D92685EF20A05A045849
:101D50008567F117BE94B7474C4593879744130A9C
:101D600044005CD85285230C0402A30104042326FA
:101D7000040223280404232A0404EFE08FFA130545
:101D80008401EFE00FFAA947232C0404F19800C85E
:101D90001CCC40D023220404232E040401469715B2
:101DA00000009385E5B12685EFE0CFF208C073709F
:101DB000043017E901001309A9798327090097E482
:101DC00001009384A47A91C798409C407C43850786
:101DD0007CC317E70100130767781C43850797E664
:101DE000010023ADF6769C40C9C38327090097F90B
:101DF00001009389E98881EB9C40DC5789E797E7EC
:101E0000010023A5877697E70100938767739843BE
:101E100097E60100938606745C549442050717E622
:101E20000100232FE67038C463F6F60017E70100BF
:101E30002322F772139527003E950A05D2854E9509
:101E4000EFE08FEE8327090081C79C40FC43DDE76C
:101E50008327090091C39C40EF10F0498547630533
:101E6000F50C59E17370043001A097E7010023AF2E
:101E7000876E1843854797F9010093896980E314B9
:101E8000F7F8CE8A17FB0100130B0B8C5685D10A8D
:101E9000EFE0EFE7E31C5BFF17F501001305C58AD0
:101EA000EFE0EFE697FA0100938A4A8B5685EFE060
:101EB0000FE617F501001305A58BEFE04FE517F5C9
:101EC00001001305258CEFE08FE417F501001305E1
:101ED000A58CEFE0CFE397E7010023A7676997E7B9
:101EE000010023A1576905B7F2406244D244424938
:101EF000B249224A924A024B05618280984094403E
:101F00007C43FD177CC3FC42A1F77360043089B7A2
:101F10006244F2404249B249224A924A024B268523
:101F2000D24405616F20E02873700430FD5717E735
:101F300001002325F760624497E7010023AAA76008
:101F4000F240D2444249B249224A924A024B97E7B0
:101F5000010023A3076005616FE0AFB47370043024
:101F600097E7010023A6075E6FE0EFC117E70100C6
:101F70001307875C1C4385071CC382807370043081
:101F800097E701009387C75C984305E317E70100D3
:101F90001307875C08439C4381CB97E70100938735
:101FA000E75C9843784301EF828017E7010013074D
:101FB000E75B14431843F8420507F8C2C1BF9843D2
:101FC00094437C43FD177CC3FC42F9FF73600430EB
:101FD0008280411106C622C4EFE02FCF97E70100AF
:101FE000938787578043EFE0EFCDB24022852244AC
:101FF0004101828097E7010093874756884382809A
:10200000797106D622D426D24AD04ECE52CC56CAA8
:102010005AC85EC697E70100938707529C43B1EF09
:1020200017E70100130747531C43850797E6010094
:1020300023A4F652832A0700638F0A0697E701005C
:102040009387C74F9C43814463F1FA0897E90100E5
:102050009389096317EA0100130A4A5183270A008A
:102060008546D85793172700BA978A07BE9983A742
:10207000090063FFF600854421A897E701009387D4
:10208000E74C9C438144850717E701002320F74C68
:1020900097E701009387474B9C4391C38544B25017
:1020A0002254268502599254F249624AD24A424B3E
:1020B000B24B4561828017E401001304E44A1C40DE
:1020C0009C43DDC37370043001A017E401001304C6
:1020D000A44997E901009389A95A17EA0100130A54
:1020E000EA4817EB0100130BEB461C409C43B5C3B9
:1020F0001C40DC4703A9C70083274900930B490014
:102100005E8563EEFA04EFE0AFC68327890213050C
:10211000890199C3EFE0CFC58327C90203270B00CC
:10212000DE85139527003E950A054E956376F700E8
:1021300017E701002320F742EFE00FBF83270A00D3
:102140000327C902DC57E362F7FA1C4085449C432D
:10215000C5F3FD5717E701002322F73E01B717E744
:102160000100232DF73CDDBD17E701001307873F72
:102170001C40184397E6010023A8E63E17E701003C
:102180002322F73E97E701009387C73B9C438507CF
:1021900017E701002328F73A1C409C4399E7FD57B5
:1021A00017E70100232CF73851BD1C40DC47DC4702
:1021B000DC4317E701002323F73849B597E701000F
:1021C00093878737984301E77370043001A00111AA
:1021D00006CE22CC26CA4AC84EC652C456C25AC0DF
:1021E0007370043097E4010093848436984061EB67
:1021F00098437D1797E6010023A0E6349C43D9EB72
:1022000097E70100938787359C43C9C797EA010088
:10221000938A0A4717EA0100130ACA3317E9010033
:102220001309C934854919A83385EA00EFE0CFAF17
:10223000832709005854DC576379F70483A70A0FF2
:10224000C1CF83A7CA0FC04713058401EFE04FB287
:10225000130B44005A85EFE0AFB15C5483260A00AB
:10226000DA85139527003E950A052A875695E3FDE2
:10227000F6FA17E70100232FF72CEFE0EFAA8327E8
:1022800009005854DC57E36BF7FA97E7010023ADD8
:10229000372B6DB701449C4081CB97E701009387B2
:1022A000E72C9C43FC4395E72285F2406244D244EC
:1022B0004249B249224A924A024B0561828017E79D
:1022C00001001307A72A14431843F8420507F8C270
:1022D00005B7EF40E04BC9BF17E401001304042722
:1022E0001C4095C31C40054999CF193B09C597E788
:1022F000010023AB27251C40FD1717E7010023270A
:10230000F7241C40FDF397E701009387E7239843E8
:102310008547E311F7F8EFE06F8F0544ADBF11CDAE
:1023200081E57370043001A017E701001307C7208F
:102330001C4399C77370043001A07370043001A06E
:10234000411122C406C614431841850617E6010050
:102350002324D61E97E60100938606209442330478
:10236000B70000C163F7E602637FE40063FD860007
:1023700097E701009387871F88431105EFE04F9F80
:102380002285EF40A03A1D3D01C9B24022444101DF
:102390008280E36FE4FCD9BF2244B24041016FE088
:1023A000EF8611C917E70100130707191C4391C7EE
:1023B0007370043001A06FE06F85411106C622C41E
:1023C0001843AA87050797E6010023A7E61697E6B4
:1023D00001009386A61917E701001307E7171843B2
:1023E00088423304F7001105EFE08F982285EF4013
:1023F000E033E93311E52244B24041016FE00F813F
:10240000B240224441018280411122C406C697E7AE
:102410000100938767129C430144850717E7010079
:10242000232CF71097E70100938747139C4363E041
:10243000F51217EE0100130E6E3097E20100938241
:10244000622301440147854F1303500A21A0311E26
:10245000638DC20B83278EFFBA86F5DB8327CEFF01
:10246000DC43232EFEFE638AC70F03AFC700DC43A5
:102470002A97814E232EFEFE6385C70783A8C700D7
:1024800093874803232017015CC383A7880423266E
:10249000F7011CC783A7C8021CCB83A70805232C00
:1024A00007005CCB03A80803834708006390670418
:1024B000C287850783C60700B3850741E38B66FEA5
:1024C0008981C205C181231EB700850E130707024B
:1024D00063061F038327CEFFDC43232EFEFEE39F0C
:1024E000C7F983274E00232EFEFE49BF8145231ED8
:1024F000B700850E13070702E31E1FFD769413171E
:102500005400311EBA86E397C2F597E7010093871E
:10251000A70503AE070083270E00639D070E97E70C
:1025200001009387270403AE070083270E00639200
:10253000071817EE0100130EAE1483274E109DE30B
:1025400083278E116395072019C223200600BD3111
:102550002285B24022444101828083274E00232EEF
:10256000FEFE21B783278E1017EF0100130F0F22F5
:10257000DC4317E701002329F7206380E73383A2B8
:10258000C700DC43AA96814E17E70100232EF71EF1
:10259000914F1303500A6388E70783A8C700938706
:1025A000480323A01601DCC283A7880423A6F601F2
:1025B0009CC683A7C8029CCA83A7080523AC060053
:1025C000DCCA03A80803834708006391672AC2870F
:1025D000850703C70700B3850741E30B67FE93D761
:1025E0002500C207C183239EF600850E938606024E
:1025F0006386122983278E10DC4317E70100232509
:10260000F718E39CE7F983270E1117E70100232D44
:10261000F71661B783274E00130F8E00D443232291
:10262000DE006388E629B307E500D84283A2C6002E
:10263000814E2322EE00894F1303500A6306EF06F2
:102640008328C7001387480323A01701D8C303A713
:10265000880423A6F70198C703A7C80298CB03A74D
:10266000080523AC0700D8CB03A8080303470800DC
:102670006318671C4287050783460700B3050741B7
:10268000E38B66FE13D7250042074183239EE700B4
:10269000850E93870702638D121B83264E00D84256
:1026A0002322EE00E31EEFF80327CE002322EE00E4
:1026B00041BF83274E00130F8E00DC432322FE0010
:1026C0006384E71F83A2C700DC43AA96814E2322BE
:1026D000FE00894F1303500A6306FF0683A8C70054
:1026E0009387480323A01601DCC283A7880423A68E
:1026F000F6019CC683A7C8029CCA83A7080523AC21
:102700000600DCCA03A80803834708006396671025
:10271000C287850703C70700B3850741E30B67FE40
:1027200093D72500C207C183239EF600850E9386AA
:102730000602638B120F83274E00DC432322FE0028
:10274000E31EFFF88327CE002322FE0041BF83272C
:10275000CE1197EE0100938EAE04DC4317E7010023
:10276000232EF7026384D71383AFC700DC433307FC
:10277000D500014397E6010023A2F6020D4F8942DE
:102780009308500A6387D707C8479307450308C3D0
:102790005CC33C452326E7011CC75C551CCB1C557C
:1027A00099C3232657003C49232C07005CCB032800
:1027B00005038347080063951705C287850783C60D
:1027C0000700B3850741E38B16FF93D72500C207A7
:1027D000C183231EF700050313070702638AAF02B4
:1027E0008327CE11DC4397E6010023A9F6FAE39D87
:1027F000D7F983274E1297E6010023A1F6FA69B7AD
:102800008147231EF700050313070702E39AAFFC75
:102810001A94E31C06D225BB8147239EF600850E41
:1028200093860602E39912F117EE0100130E4EE5AE
:1028300083274E10769493165400E38307D01DB37C
:102840000147239EE700850E93870702E39712E571
:1028500097E70100938707D103AE0700769493169C
:10286000540083270E00E38607CCA1B58147239E41
:10287000F600850E93860602E39E12D783278E11FB
:10288000769493165400E38107CCD1B583274E127A
:1028900017E701002324F7F0C1BD83270E1117E7C6
:1028A00001002323F7EEE1B98327CE002322FE00A7
:1028B00011BD8326CE002322DE00B5B3797126D266
:1028C0004AD04ECE52CC56CA5AC85EC606D622D47C
:1028D00097E90100938949C617E90100130949DA0C
:1028E00017EA0100130ACAC697EA0100938A0AC8C8
:1028F00097EB0100938B8BC697E40100938444C649
:10290000054B21A883A7090003244910850717E771
:1029100001002323F7C25D3011E89C40E5F78327CF
:102920000900E37CFBFEEFD07FAEC5BF73700430BF
:1029300083270A00B9E383270911C0471305440020
:10294000EFD01FC383A70B00FD1717E70100232754
:10295000F7C09C40FD1717E701002323F7C083272A
:102960000A0089C783A70A00FC4385E30858EF10D3
:1029700050042285EF10F0034DB703A70A0083A788
:102980000A007C4385077CC37DB703A70A0083A6A2
:102990000A007C43FD177CC3FC42E9FB73600430F2
:1029A000F1B797E70100938727B99C43DDE7411111
:1029B00006C622C426C297E7010023A707B817E777
:1029C00001001307A7BA1C43B7A6A5A59386565ABC
:1029D0009C5B8C43639BD500D0436318B60094473F
:1029E0006395C600DC476388D70008430C43938592
:1029F0004503EF20C07317E701001307A7B5144381
:102A000017E401001304C4C711A81C43A9CF1C4339
:102A1000FD1797E6010023AFF6B214439397260003
:102A2000B6978A07A2979C43EDD3084393172500D6
:102A3000AA978A073307F4005443A107A297C44218
:102A400044C36385F402DC44B240224417E701002A
:102A5000232EF7B0924441018280854717E7010099
:102A60002324F7AE82807370043001A0C440D145A6
:102A7000EF30503E229544C1F9B701114AC806CE45
:102A800022CC26CA4EC62A897370043097E401000E
:102A9000938404AC9C4017E40100130424ADD9E7EF
:102AA0006314090003290400930949004E85EFD0FF
:102AB0003FAC8327890289C713058901EFD05FAB3B
:102AC000CE8517E50100130525CDEFD0FFA59C406D
:102AD00081C71C40FC43ADE31C40638B27079C402F
:102AE0009DCF737004309C40C1EB97E70100938742
:102AF000A7A79843184325EBFD5717E70100232F9D
:102B0000F7A29C4089CF1C40FC4391CB1840144055
:102B10007C43FD177CC3FC4299E373600430F240B0
:102B20006244D2444249B2490561828018401C4047
:102B30007C4385077CC3ADB7184014407C43FD1728
:102B40007CC3FC42D1FB736004301C40E39927F93D
:102B50009C40A1C397E701009387079E9C43ADCBA0
:102B60007370043001A09C43DC47DC47DC4317E76B
:102B700001002325F79C71B718401C407C43850752
:102B80007CC397E701009387279E984318432DD76E
:102B9000D9BF97E701009387679C17E701001307E8
:102BA00027AE9C4303278711631DF700F240624460
:102BB00097E7010023AC079AD2444249B249056124
:102BC00082806244F240D2444249B2490561D1BB9D
:102BD0006244F240D2444249B24905616FD01F833A
:102BE0003DC9411126C297E40100938424984AC04C
:102BF0002E898C4006C622C4E105EFD07F94884020
:102C00001105EFD0FF96FD57630AF90497E701001D
:102C100093878794804398409C434A9440C3636C55
:102C2000F40497E701009387279488438C4091052B
:102C3000EFD01F9197E70100938747909C436376FD
:102C4000F40097E7010023AB878EB2402244924400
:102C50000249410182807370043001A08C402244FB
:102C6000B2409244024917E501001305E5B291050F
:102C700041016FD07F8B97E701009387A78E884330
:102C800022448C40B24092440249910541016FD0E8
:102C90003F8B11C997E701009387078A9C4399E707
:102CA0007370043001A07370043001A0411126C27A
:102CB00097E401009384848B9840AE878C40B706DC
:102CC0000080D58F06C622C41CCFE1053284EFD028
:102CD000BF8588401105EFD0BF89FD57630EF40012
:102CE00097E70100938747878843B2409244229533
:102CF000224441016F3090238C402244B2409244E0
:102D000017E50100130545A9910541016FD0DF8149
:102D100025CD411126C297E40100938424854AC041
:102D20002E898C4006C622C4E1053284EFD0CFFF45
:102D300088401105EFD0DF838547630AF40497E7E5
:102D4000010093876781804398409C434A9440C325
:102D5000636CF40497E701009387078188438C40F4
:102D60009105EFD0EFFD97D701009387277D9C4316
:102D70006376F40097D7010023A2877CB2402244F7
:102D800092440249410182807370043001A08C405A
:102D90002244B2409244024917E501001305C59F41
:102DA000910541016FD04FF897D701009387877B3A
:102DB000884322448C40B24092440249910541012B
:102DC0006FD00FF8411106C622C426C25C45C04729
:102DD00035CC930484012685EFD08FF997D7010075
:102DE000938787759C43B5E7930444002685EFD00D
:102DF0002FF897D701009387E77558549C4363F6E3
:102E0000E70097D7010023A7E77493172700BA9725
:102E10008A0717E501001305A586A6853E95EFD024
:102E2000AFF097D70100938767749C4358540145CE
:102E3000DC5763F8E700854717D701002326F770B2
:102E40000545B240224492444101828073700430AF
:102E500001A0A68517E5010013058591EFD0CFEC01
:102E6000C9B797D701009387276D9C4381E773709B
:102E7000043001A0411106C622C426C2B707008053
:102E80004045CD8F1CC12DC4EFD08FEE930444007C
:102E90002685EFD0EFED97D701009387A76B5854A5
:102EA0009C4363F6E70097D7010023A5E76A9317D1
:102EB0002700BA978A0717D501001305657C3E9550
:102EC000A685EFD06FE697D701009387276A9C43CA
:102ED00058540145DC5763F8E700854717D70100D0
:102EE0002324F7660545B240224492444101828082
:102EF0007370043001A011CD97D7010093878764C8
:102F0000984397D70100938727659C4318C15CC1FC
:102F100082807370043001A055C1D1CD411106C625
:102F200022C42A877370043097D8010093884862BE
:102F300083A7080091CB97D7010093872763944319
:102F40009C43FC428507FCC217D301001303C360F6
:102F50009C4103260300FD560144638FD70217DE10
:102F60000100130E2E5E03250E00032807005443B4
:102F70006305A80005446371D6023308D6400544B2
:102F8000637CF80003250E00918F03260300B6979B
:102F90009CC108C350C3014483A7080081CB97D7C5
:102FA00001009387A75C9C43FC4381EF2285B240DC
:102FB0002244410182807370043001A07370043098
:102FC00001A0EF30E07CDDB7854717D70100232D46
:102FD000F756828019C1684582800145828011C1FF
:102FE0006CC5828097D701009387475888438280B9
:102FF00097D701009387C7559C43054589CB97D741
:1030000001009387675388431335150006058280B6
:1030100031CD011126CA97D40100938424559C40D8
:1030200006CE22CC4AC84EC65855DC576379F70203
:103030001C4D63C707009C40D457A947958F1CCDF2
:1030400093172700BA97584917D901001309496304
:103050008A07CA97630DF7009C40DC575CD5F240A5
:103060006244D2444249B249056182808280930918
:1030700045002A844E85EFD0AFCF9C4017D7010082
:103080001307474D1843DC575CD46376F70017D716
:1030900001002321F74C139527003E9562440A0551
:1030A000F240D244CE854A95B249424905616FD07B
:1030B000AFC719CD411106C622C426C297D7010059
:1030C0009387C74A80436307A4007370043001A04C
:1030D000014582807C4881E77370043001A054541C
:1030E0003848FD177CC86383E60099C70145B240A4
:1030F0002244924441018280930444002685EFD00B
:103100002FC7284897D701009387C7449843A947FA
:10311000898F48D41CCC6376A70097D7010023ABD6
:10312000A742D145EF30005397D701009387475509
:103130003E95A685EFD04FBF054555BF737004304F
:1031400097D701009387C7409C4391CB97D7010045
:103150009387C74198439C437C4385077CC3828007
:1031600097D701009387C73E9C438DC397D7010033
:103170009387C73F9843784311CB984394437C434C
:10318000FD177CC3FC4299E373600430828097D7BB
:1031900001009387A73D904394439843A947D45691
:1031A000084E958F1CCF828097D701009387073CEC
:1031B000984309C79443F84A0507F8CA88438280B0
:1031C00079714AD006D622D426D24ECE2A8973707F
:1031D000043097D401009384A4379C4017D4010095
:1031E0001304C438BDE31C40BC4F89E71C400547AD
:1031F000F8CFD1E19C4081C71C40FC43F1EB7370D8
:1032000004309C408DEF1C40A84F11C56304090297
:103210001C4023AC07041C4023AE07049C4081C71C
:103220001C40FC438DEBB250225492540259F24997
:103230004561828018403C4FFD173CCFE9BF1840E4
:103240001C407C4385077CC37DBF18401C407C43E9
:1032500085077CC349BF184014407C43FD177CC3DD
:10326000FC42F1F373600430B2502254925402597C
:10327000F2494561828008402EC61105EFD04FAF5C
:10328000B245FD576380F50697D701009387C72C99
:1032900083A9070018409C43AE992322370163ECB1
:1032A000F90497D701009387272C88430C40910598
:1032B000EFD00FA997D70100938747289C4363F667
:1032C000F90097D7010023AB3727EFD02F941DB714
:1032D000184014407C43FD177CC3FC428DF373609F
:1032E000043031BF0C4017D501001305E54A9105A4
:1032F000EFD08FA3D9BF97D701009387A726884324
:103300000C409105EFD0CFA3C9B779714AD04ECE0A
:1033100006D622D426D252CC2E89B28973700430BC
:1033200097D401009384C4229C4017D40100130455
:10333000E423F9EF18408947784F630CF7001C40ED
:103340001345F5FFB84F798DA8CF1C400547F8CF3E
:10335000ADE69C4081C71C40FC43F5E3737004302C
:103360009C40B1E7638609001C40BC4F23A0F900D4
:10337000184085470145784F630BF7001C401349FF
:10338000F9FF0545B84F3379E90023AC27051C4008
:1033900023AE07049C4081C71C40FC43C1E3B250EC
:1033A000225492540259F249624A4561828018407F
:1033B0001C407C4385077CC375B7084036C61105A1
:1033C000EFD00F9BB246FD576385F60897D70100F3
:1033D0009387871803AA070018409C43369A232234
:1033E00047016363FA0897D701009387E71788437B
:1033F0000C409105EFD0CF9497D701009387071425
:103400009C436370FA0697D7010023A9471391A83C
:1034100018401C407C4385077CC329BF18401440DA
:103420007C43FD177CC3FC42BDFB73600430B2508B
:10343000225492540259F249624A456182801840EE
:1034400014407C43FD177CC3FC4289FB736004304D
:1034500031B70C4017D50100130505349105EFD0A5
:10346000AF8CEFC0BFFAF5B597D701009387870FF0
:1034700088430C409105EFD0AF8CE5B751C14111A5
:1034800006C622C426C24AC07370043097D4010015
:103490009384040C9C40B9EB99C23C4D9CC2B2870A
:1034A0008946704D74CD2E872A846386D70663FCC7
:1034B000F6048D456387B70091456395B7006300B7
:1034C000D60C38CC8547630FF60405449C4081CB6D
:1034D00097D70100938787099C43FC43A9E3228582
:1034E000B2402244924402494101828097D70100B0
:1034F0009387C70798439C437C4385077CC369BF78
:103500007370043001A08546E39ED7FA3C4D33E743
:10351000B70038CD45BF3C4D85073CCD65B7EF3092
:10352000202775BF130944004A85EFD06F8497D7D1
:1035300001009387270248549C4363F6A70097D75E
:10354000010023A9A700D145EF30C01097D7010093
:10355000938707133E95CA85EFC01FFD1C5481C792
:103560007370043001A097D70100938727009C4314
:103570005854DC57E3FBE7F4EFC05FE9B9B7014407
:10358000B1B739CD011122CC26CA4AC84EC652C4A1
:1035900056C206CEBA89368AB2842E892A84EFC0F2
:1035A000DFF2AA8A63050A003C4C2320FA00784C1B
:1035B00089477CCC6389F40263F4970C8D4663875A
:1035C000D40091466396D400630AF70A232C24059D
:1035D0008547631EF7061C5499CB7370043001A015
:1035E0007370043001A03C4C85073CCCD5B797D70D
:1035F0000100938767F49C43ADEB93044400268558
:10360000EFC01FF797D701009387C7F448549C4336
:1036100063F6A70097D7010023AEA7F2D145EF309C
:10362000600397D701009387A705A6853E95EFC055
:10363000BFEF97D70100938767F39C435854DC573B
:1036400063F7E70063850900854723A0F900054477
:103650005685EFC03FE72285F2406244D24442499A
:10366000B249224A924A056182809305840117D5A6
:1036700001001305E50FEFC03FEB65BF0144C9BF73
:103680008547E397F4F43C4C33E92701232C2405C8
:1036900081B74DC1011122CC26CA2A844EC606CE5E
:1036A0004AC8AE84EFC07FE28947744C7CCC3C4C66
:1036B0000547AA8985073CCC6395E6061C5481C75B
:1036C0007370043001A097D701009387E7E69C430D
:1036D000ADE7130944004A85EFC09FE997D7010081
:1036E000938747E748549C4363F6A70097D70100A8
:1036F00023A2A7E6D145EF20F07597D70100938765
:1037000027F8CA853E95EFC03FE297D7010093871F
:10371000E7E59C435854DC5763F5E70099C08547BB
:103720009CC06244F240D24442494E85B249056190
:103730006FC05FD97370043001A09305840117D561
:1037400001001305E502EFC03FDEC1B7AA8729C516
:103750007370043017D70100130787DF14439DE20D
:10376000F04F894601456315D60023AE0704054591
:103770001C4381CB97D70100938747DF9843784359
:1037800015E3828097D60100938646DE90429442EC
:103790007442850674C2E9B797D70100938707DDA5
:1037A0009C437DB7984394437C43FD177CC3FC4204
:1037B000E9FB7360043082805D71A6C2CAC052DC2E
:1037C00056DA5AD85ED686C6A2C44EDE62D466D217
:1037D0006AD017D90100130969DA17DB0100130B4E
:1037E0002BD997D401009384E4D897DA0100938A07
:1037F000AAD8054AA54B83270900984363010712FD
:10380000DC4783A90700EFE06FF6EFE02FF783278F
:103810000B002A8C6362F50A97D7010023AAA7D46C
:1038200001466370351B8840B3858941EFD0DFBD09
:10383000EFE0DF98630105128840814601462C00C5
:10384000EFD0EFEB4DD9A247E3C807FEC24983A7EB
:10385000490189C713854900EFC09FD1EFE00FF2FE
:1038600083270B002A8C636DF508A24717D7010048
:10387000232087D1E3E2FBFCB317FA0013F70721FB
:10388000631A071613F7770C6318071E93F70702DE
:10389000C5D74E85EF00F01145B7DC47C04783AC74
:1038A0000700930944004E85EFC09FCC5C502285F1
:1038B00082975C4C6384470B83270900984371FF10
:1038C00003A70A0097D6010023A486CB97D6010050
:1038D00023A4F6CA97D7010023A2E7CAEFE01F8E00
:1038E000A1BFDC47C04703AD0700930C44006685C9
:1038F000EFC01FC85C50228582975C4C63864709E5
:1039000083270900984371FF03A70A0097D6010097
:1039100023A4F6C697D7010023A2E7C6B9B7EFE004
:10392000EFE4EFE0AFE583270B002A8CE366F5F8C0
:1039300083A70A00884081499043B385894117D7FE
:103940000100232787C313361600EFD0FFABEFE04B
:10395000FF86E31305EEEFC07FABF9BD1C4CCE85AF
:10396000E69763E9FC049C4089CF02CA66CC22CE6C
:10397000EFF00FE88840814601464C08EFC03FE277
:1039800005FD7370043001A01C4CE685EA97636C5A
:10399000FD049C4089CF02CA6ACC22CEEFF04FE5ED
:1039A0008840814601464C08EFC07FDF31F97370D3
:1039B000043001A0032509005CC000C8EFC05FB857
:1039C000E5BDEFE0AFFF83270900DC47C047930C5C
:1039D00044006685EFC0DFB95C4C638F47035C50E1
:1039E0002285829791BD032509005CC000C8EFC005
:1039F0003FB539B7B24723ACF900A5CFE29723A270
:103A0000F90023A8390193854900636FFC0403A5DD
:103A10000A00EFC0FFB20DB51C4C00C83387F90097
:103A200058C0636DEC02330C3C416363FC029C4064
:103A300089CF02CA4ECC22CEEFF08FDB8840814680
:103A400001464C08EFC0BFD559F97370043001A08E
:103A500003A50A00E685EFC0BFAE51B703250900F4
:103A6000E685EFC0FFADA5BF03250900EFC05FAD40
:103A7000E1B37370043001A0B24783A6890123A883
:103A800039013387D70023A2E9006364EC04B3074C
:103A9000FC4063EBD70483A749024E85829783A736
:103AA000C901E39B47D983A68901B2479840B697DD
:103AB00011CF02CA3ECC4ECEEFF08FD38840814664
:103AC00001464C08EFC0BFCDE31805D67370043033
:103AD00001A06374FC00E370F7FC032509009385E3
:103AE0004900EFC0FFA589BB03A50A0093854900E3
:103AF000EFC01FA591B3411122C406C626C24AC019
:103B000017D40100130404A7EFF04FE31C4095CB3A
:103B1000EFF00FE51C409DC38148014881470947EC
:103B200081461306004097D5010093852589170526
:103B300000001305A5C8EFD05F9A39E9737004300F
:103B400001A017D90100130969C64A85EFC03F9C3F
:103B500097D401009384C4C62685EFC05F9B0146BD
:103B6000B145114597D7010023AA27A197D7010096
:103B700023A497A0EFC09FB517D70100232CA79EC1
:103B800011CD97D501009385E582EFD0AFFC49B701
:103B9000B240224492440249410182807370043051
:103BA00001A0A5C9797156CAAA8A1305C00222D4F8
:103BB00026D24AD04ECE52CC06D65AC85EC63A89D4
:103BC000B689328AAE84E9212A8405C9EFF00FD77D
:103BD00097D701009387079A9C439DCFEFF04FD86A
:103BE000130544002320540104CC232E4401232038
:103BF000340323222403EFC0DF922285B2502254E3
:103C000092540259F249624AD24A424BB24B456140
:103C100082807370043001A097DB0100938B0BB995
:103C20005E85EFC0DF8E17DB0100130B6BB95A8581
:103C3000EFC0FF8D0146B145114597D7010023AF75
:103C4000779397D7010023A96793EFC03FA817D7B1
:103C500001002321A79201C997C5010093858575AD
:103C6000EFD04FEFA5BF7370043001A039C501112B
:103C700022CC06CE26CA17D401001304A48F8328B1
:103C800004002A88014563850802BA842EC236875B
:103C900032C442C6954663C5B602EFF06FB5894798
:103CA000630BF5020840814601464C00EFC03FAF70
:103CB000F2406244D244056182807370043001A0F6
:103CC0004C0081463A864685EFD0EF87F240624449
:103CD000D244056182800840814626864C00EFC0B0
:103CE0001FACF9B719C1084182807370043001A07C
:103CF00001E57370043001A0411106C622C42A8474
:103D0000EFF0CFC348483334A000EFF06FC52285F1
:103D1000B24022444101828001E57370043001A069
:103D2000411122C42A8406C6EFF04FC10050EFF0C3
:103D30002FC3B240228522444101828001E5737085
:103D4000043001A0411122C426C22E84AA8406C6D2
:103D5000EFF0CFBE80D02244B240924441016FF0D8
:103D60002FC04111714522C406C61D262A8411C5E3
:103D7000232005001105EFC08FF92285B2402244AF
:103D80004101828001CDB70700FFED8F81C77370BD
:103D9000043001A099E57370043001A07370043001
:103DA00001A0011122CC4AC84EC652C456C206CE4A
:103DB00026CABA893689B28A2E842A8AEFF04FA39E
:103DC00011E5638509007370043001A0EFE00F9ADC
:103DD00083240A00B37794006316090295C76387AA
:103DE0000A009347F4FFE58F2320FA00EFE00FBDB0
:103DF000F240624426854249D244B249224A924A5C
:103E000005618280E30DF4FCE38209FEB3355001C5
:103E1000E20563050900B7070004DD8D4E86C18DFC
:103E200013054A00EFE0FFE6EFE04FB919E1EFC0FC
:103E3000EFDDEFF0CFB593176500AA8963D80700CF
:103E4000B7040001FD14B3F499005DB7EFF00FAFB4
:103E500083290A00B3773401631E090089CB638884
:103E60000A009347F4FFB3F737012320FA00EFF07D
:103E70002FAFF9B7E31DF4FEDDB701C9B70700FFA7
:103E8000ED8F99C77370043001A07370043001A0E6
:103E9000411122C42A8406C626C24AC02E89EFF0E8
:103EA000EFA904409345F9FFB3F795001CC0EFF06C
:103EB0002FABB240224426850249924441018280C0
:103EC000411122C42A8406C6EFC02FE00040EFC093
:103ED0006FDFB240228522444101828009C9370741
:103EE00000FFB3F7E50099C77370043001A0737049
:103EF000043001A06F20900BB70700FFF18F81C73E
:103F00007370043001A001E67370043001A0011148
:103F100022CC4AC84EC652C406CE26CA3689AE89BD
:103F20002A8A3284EFF0CF8C21E163050900737097
:103F3000043001A0EFE08F8383240A00CE855285F0
:103F4000B3E49900613FB37794006307F4068324D8
:103F50000A00EFE0AFA6F240624426854249D2440F
:103F6000B249224A05618280EFE04F8083240A0033
:103F7000CE855285B3E434019537B3F78400638D61
:103F80008702E30609FCB70500054A86C18D1305C3
:103F90004A00EFE01FD0EFE06FA219E1EFC00FC7BA
:103FA000EFF0EF9E93176500AA8463DF0700B70761
:103FB0000001FD17FD8C45B783270A001344F4FF69
:103FC000E18F2320FA0071B7EFF04F9783240A00A6
:103FD000B3779400639787009347F4FFE58F23201E
:103FE000FA00EFF0EF97E1B7411122C406C62A8428
:103FF00026C2EFD0BFF75C4085C308489304C400D5
:104000006316950015A0084863009502B7050002E5
:10401000EFE03FE55C40E5FB2285612A2244B240A7
:10402000924441016FE08F997370043001A009C977
:10403000370700FFB3F7E50099C77370043001A09C
:104040007370043001A06F20607601C9B70700FFCC
:10405000ED8F99C77370043001A07370043001A014
:10406000411122C426C206C62A84AE84EFF00F8D09
:10407000184093C7F4FFF98F1CC02244B240924409
:1040800041016FF0EF8D19C1084D8280014582809A
:10409000411122C406C62A84EFD05FED97C7010004
:1040A0009387074E9C43A1EBE56717C701001307F1
:1040B000A772F11797C6010023AAE64C17C70100A3
:1040C0002324F74C17C70100232AF77097C7010074
:1040D0009387474B17C701002320F770854717C701
:1040E00001002327074A17C70100232D074817C7D8
:1040F00001002327F74819E8EFE04F8CEF10A002EA
:1041000001442285B240224441018280130584008B
:1041100093773500C1EFE5671307F5FFE917E3ED86
:10412000E7FC97C60100938666469C4229A0984307
:1041300011C7BE86BA87D843E36BA7FE17C7010035
:1041400013074744E38AE7FA9843414613848700FC
:1041500098C2D843B306A7406378D6023388A70035
:104160002322D800C8C38325480097C60100938640
:10417000E64111A0BA8698425043E36DB6FE232073
:10418000E80023A00601D84397C70100938747435F
:104190009C43998F17C701002324F742EFE00F8259
:1041A00031DC2285B240224441018280719911059F
:1041B0009DB729C9411122C406C62A84EFD01FDB4E
:1041C000930584FF0326C4FF17C701001307073CAC
:1041D00011A03E871C43D443E3EDC6FE232CF4FE1E
:1041E0000CC397C701009387A73D98438327C4FF5B
:1041F0002244B240BA9717C701002323F73C41017C
:104200006FD0DFFB828097C701009387673B8843AD
:10421000828082803367B5000D8BAA871DE79308E3
:10422000D6FFAA982A87AE866371150303A80600F5
:1042300011079106232E07FFE36A17FF9347F5FF47
:10424000C697F19B9107BE95AA972A9663F3C70A72
:104250009386450013884700B3B6D70033B80501ED
:1042600033E7F50093C61600134818000D8BB3E62C
:10427000060113371700758F330EF640938617002B
:1042800029CF1337AE0031EB13532E002E88BE8694
:104290000147832808000507110823A0160191068D
:1042A000E36967FE1377CEFFBA95BA976302EE040F
:1042B00083C60500138717002380D700637AC702DF
:1042C00083C6150013872700A380D7006372C70237
:1042D00003C725002381E7008280B307F640AE972D
:1042E000850503C7F5FF8506238FE6FEE39AF5FEF5
:1042F00082808280B367C5008D8BB308C500E9C397
:104300006371150FB307A0408D8B13873700954657
:1043100093F5F50F130815003383A8407D166373DA
:10432000D70015476363E60CD5CF2300B5000547DA
:10433000638DE700A300B5000D47130825006396C1
:10434000E700130835002301B500139685004D8E54
:1043500013970501518F3303F34093968501D98E4E
:1043600013562300AA97014794C305079107E36DED
:10437000C7FE1377C3FFB307E8006307E306238094
:10438000B70013871700637C1703A380B700138758
:104390002700637617032381B70013873700637004
:1043A0001703A381B70013874700637A170123829D
:1043B000B7001387570063741701A382B700828088
:1043C00093F5F50F13978500D98D139705014D8F40
:1043D000E37715FFAA87910723AEE7FEE3ED17FF0A
:1043E000828082802A8895B78280AA8749BF8347C6
:1043F00005002A8799C7050583470500EDFF198D3C
:1044000082800145828005058347F5FF850503C746
:10441000F5FF91C7E389E7FE3385E7408280814756
:10442000E5BFAA87850503C7F5FF8507A38FE7FECC
:1044300075FB828083460500930700026397F600B0
:10444000050583460500E38DF6FE938756FD93F739
:10445000D70F85C7AA87814585CE01458507138675
:1044600006FD1317250083C607003A950605329509
:10447000F5F699C13305A0408280938536FD8346C9
:10448000150093B5150093071500E1FA0145D5B75E
:10449000014582809C412380A7009C4185079CC1E7
:1044A000828097C601009386E60E9C421757030050
:1044B0001307473513861700BA972380A70097C5BF
:1044C000010023A9C50CA9476308F5009307000460
:1044D0006305F6000145828075DE370610F005079A
:1044E0008347F7FF2320F6F09C42FD1797C5010094
:1044F00023A2F50AEDF7014582804D712322911424
:1045000023202115232A5113232481132326111438
:1045100023248114232E3113232C411323286113C8
:1045200023267113232291132320A113232EB111CB
:10453000AA842E8932C6130C5002A54A834709006B
:1045400063808703B9CB804011A0A1CB2300F40086
:1045500080400509050480C083470900E39787FF71
:104560000346190093081900C686130D0002FD5971
:104570007D5A0148130550059307D6FD93F7F70FB1
:10458000138916006363F52A17C70100130787A76D
:104590008A07BA979C43BA9782878320C114032461
:1045A000811483244114032901148329C113032A8C
:1045B0008113832A4113032B0113832BC112032C74
:1045C0008112832C4112032D0112832DC1117161BF
:1045D0008280A14C02C4854763D50715B24780404D
:1045E000938B770093F68BFF03AB060083A94600FD
:1045F000938786003EC6668681465A85CE85EF1033
:1046000070352AC8814763853723930D4101854B57
:10461000668681465A85CE85EF10005681466686AD
:104620002A8BAE89EF101033A24723A0AD009386EA
:104630001B00910D63843701B68BD9BFE37E9BFFCE
:1046400063DD4601A2872380A70180407D1A93077E
:1046500014009CC03E84E3C846FF93962B001C08C0
:10466000BE9631A8938777052300F4008040FD1B98
:1046700093871B00050480C0F116E351F0EC9C42C7
:10468000E3E2FAFE93870703C5B79C409306000355
:1046900032472380D7009C4093064700C14C1386C5
:1046A000170090C013068007A380C700804002C493
:1046B000BA87050480C003AB0700814936C625BF11
:1046C000B24783AC0700938B470063840C1C635F85
:1046D00040199307D0026319FD1683C70C0085C3E8
:1046E00063DC09189440850C7D1A2380F600804015
:1046F000050480C083C70C00E5F7635D400180407E
:10470000930700022300F40080407D1A050480C056
:10471000E31A0AFE5EC61DB502C48547A94CE3CF65
:1047200007EBB24780409386470071B703C6160077
:10473000CA8699B59C40930650022380D7008040DA
:10474000050480C0E5BBC14C02C471B5B24703C6C5
:104750001600CA8683A9070091073EC6E35E0AE0F9
:104760004E8AFD5911BD03C61600130DD002CA862C
:1047700021B59347FAFFFD8703C61600337AFA0086
:10478000CA86DDBB03C61600130D0003CA86EDB34F
:1047900083C51600930906FDCA86938705FD2E86FC
:1047A000E3EEFAFA93972900BE9985068609AE9939
:1047B00083C50600938909FD938705FD2E86E3F3E3
:1047C000FAFE69BF32479C40144311073AC6238062
:1047D000D7008040050480C095B3854763D3070B9D
:1047E000B24793867700E19A938786003EC683A9F5
:1047F00046009C4263DC090A94401306D002B307CA
:10480000F0402380C6008040B336F000B309304149
:10481000050480C03E8BB389D940A94C02C4E1BBDA
:1048200003C616000508CA8681BB9C40468921B78D
:10483000E37D9BDD8547814B8546E3C547E131BD7F
:1048400097CC0100938C0CB8CE856685EF00105B89
:10485000330AAA40635C400180402300A4018040E9
:104860007D1A050480C0E31A0AFE014A83C70C00C2
:10487000E38207EAE3C809E6FD197D57E394E9E618
:10488000ADBDB247938647009C4336C693D9F741E6
:1048900095B7635640019307D002E313FDFA97CC16
:1048A0000100938C2CB2930780021DBD3E8BA94C56
:1048B00002C4804089B34D71232E3113B7090040E3
:1048C0009387F9FF2324811423229114232C41136D
:1048D000232A511323261114232021152328611381
:1048E0002326711323248113232291132320A11340
:1048F000232EB1112A8A2EC417C40100130484C9BF
:10490000975A0300938A0AF097C4010093840485A0
:104910003EC693055002294513080004B70610F05F
:1049200083470A006386B704C1C71840050A130607
:104930001700569797C8010023AEC8C42300F7009C
:104940006382A706E31E06FD17570300130787EBD4
:1049500005078347F7FF23A0F6F01C40FD1717C695
:1049600001002329F6C2EDF783470A00E39EB7FA58
:1049700083461A0013051A002A87930B00027D5BF9
:104980007D5C014893055005A5489387D6FD93F7B4
:10499000F70F130A170063E7F5348A07A6979C43BD
:1049A000A6978287175703001307C7E555F28DBFF7
:1049B0008320C11403248114832441140329011486
:1049C0008329C113032A8113832A4113032B011363
:1049D000832BC112032C8112832C4112032D01124F
:1049E000832DC11171618280A14C014D854763DB2C
:1049F0000719A2479D07E19B83AD070003AB470062
:104A0000138787003AC4668681466E85DA85EF1083
:104A100060742AC863066D351309410185496686AD
:104A200081466E85DA85EF10201566868146AA8D4F
:104A30002E8BEF1020722320A90085091109E310A5
:104A40006DFFE3FE9DFD13060004B70610F063D171
:104A500089031C4013871700D69797C5010023AB25
:104A6000E5B223807701630CC7047D1CE3C389FF93
:104A7000B2476800A548B386F9008A061C08BE96AE
:104A8000294813030004370610F0E384A6E89C428B
:104A90009305000363F4F800930570051840AE9782
:104AA00093051700569717CE01002325BEAE2300AD
:104AB000F7006380072B638C6526F116F9B717574B
:104AC0000300130727D405078347F7FF23A0F6F059
:104AD0001C40FD1797C5010023AEF5AAEDF77D1C1C
:104AE00071B71C40130600041387170097C5010017
:104AF00023A2E5AAB386FA00930500032380B6003B
:104B00006300C73E890797C6010023A5F6A85697FC
:104B1000930680072300D70017570300130787CE9B
:104B2000B70610F0639EC70005078347F7FF23A071
:104B3000F6F01C40FD1717C60100232DF6A4EDF773
:104B4000A247C14C014D91072247014B832D07001D
:104B50003EC455BDA24783AC070013894700638F4D
:104B60000C3A635480219307D002639EFB2E03C747
:104B70000C00BA856310072025AC8547A94C014D70
:104B8000E3C907E7A2479107C1B7A24783461700C9
:104B9000528703AB070091073EC4E3580CDE5A8CE2
:104BA0007D5BE5B383461700930BD0025287F1BBC0
:104BB0009347FCFFFD8783461700337CFC00528738
:104BC000E9B383461700930B000352877DBB03466E
:104BD0001700138B06FD5287930706FDB286E3EE9E
:104BE000F8FA93172B00DA9705078607B297034662
:104BF0000700138B07FD930706FDB286E3F3F8FE6B
:104C000069BFA2451C402946984193861700D69754
:104C100017C501002320D5982380E700138945009C
:104C20006301C72A930700046387F6204AC4D5B1FD
:104C3000854763DF0729A24713877700619B9307A6
:104C400087003EC4032B47001C43635B0B301840B6
:104C5000130600049306170097C5010023ACD592F4
:104C600056979305D0022300B7006388C62CB3077C
:104C7000F0403337F000330B6041BE8D330BEB4017
:104C8000A94C014D49B38346170005085287F5B971
:104C9000834617005287D5B91C409306000413873A
:104CA000170017C601002327E68ED6971306500279
:104CB0002380C700E31FD7C417570300130787B427
:104CC000B70610F005078347F7FF23A0F6F01C4056
:104CD000FD1717C60100232FF68AEDF71DB9C14C49
:104CE000014D29B31C40930600042A8A138717003C
:104CF00017C601002320E68AD697130650022380A8
:104D0000C700E318D7C0175703001307A7AFB706AC
:104D100010F005078347F7FF23A0F6F01C40FD17AE
:104D200017C601002328F686EDF72A8ADDB6175745
:104D30000300130727AD05078347F7FF2320F6F08D
:104D40001C40FD1797C5010023A6F584EDF7F11669
:104D50002DBB175703001307E7AAF1FDF11635B372
:104D6000E3FC9DCB8549C5B1014C03C70C00BA8556
:104D7000E30E07EAFD58294513080004B70610F0B2
:104D800063570B0A1C4013861700D69717C3010000
:104D90002322C3802380E7006384A50663040609F9
:104DA000850C03C70C007D1CBA8579FBE35080E9B4
:104DB0001C409305000213060004B70610F021A062
:104DC0007D1CE3050CE613871700D6972380B700F8
:104DD00017B501002320E57CBA87E313C7FE1757F8
:104DE0000300130727A205078347F7FF23A0F6F068
:104DF0001C40FD1717B50100232EF578EDF7C9B754
:104E000017570300130707A041DE05078347F7FF85
:104E100023A0F6F01C40FD1717B60100232CF676F0
:104E2000EDF7BDBF175703001307C79DF9BF7D1BE3
:104E3000E31A1BF5A5BF175703001307A79CB70676
:104E400010F005078347F7FF23A0F6F01C40FD177D
:104E500017B601002320F674EDF74AC45DBC97BC79
:104E60000100938C2C56DA856685EF002079330C8F
:104E7000AC40E35C80EF1C4013060004B70610F062
:104E800021A07D1CE3020CEE13871700D697238028
:104E9000770197B5010023AFE56EBA87E313C7FE2C
:104EA000175703001307079605078347F7FF23A04B
:104EB000F6F01C40FD1797B5010023ADF56CEDF73A
:104EC000C9B7175703001307E793B5FA4AC491B45B
:104ED000A247138747009C433AC413DBF741B5B39D
:104EE0001757030013070792B70610F0050783470B
:104EF000F7FF23A0F6F01C40FD1717B60100232B87
:104F0000F668EDF7854717B701002325F768930783
:104F10008007175703002307F78E1DB163568001E2
:104F20009307D002E39DFBF297BC0100938C8C4960
:104F3000130780029305800235BD975603009386C0
:104F4000668C370610F0850603C7F6FF2320E6F0CF
:104F500018407D1797B5010023AEE5626DF701BBE0
:104F6000BE8DA94C014D45B4B70710F023A0A7F2A0
:104F700001A03971130341022ED29A8506CE32D494
:104F800036D63AD83EDA42DC46DE1AC62D32F24038
:104F90000145216182805D711303810322D42AC6F9
:104FA00032DC2A841A86680006D6BEC236DEBAC053
:104FB000C2C4C6C61ACEEFF04FD4B2472380070052
:104FC0003245B250018D225461618280B70710F0E2
:104FD00083A647F403A607F403A747F4E31AD7FE12
:104FE0009306067D33B6C600B305E60023A4D7F4C6
:104FF00023A6B7F48280B70710F003A747F403A6EF
:1050000007F483A647F4E31AD7FE9306067D33B66A
:10501000C60023A4D7F4B305E60023A6B7F493078C
:10502000000873A047308280411122C406C697B79A
:1050300001009387A75617B401001304E455984361
:105040001C40930647069387470617B601002325A1
:10505000F654856717B601002322D654938777BB91
:1050600063C6D700B240224441018280FD77938716
:10507000C74A3E9797B7010023A2E7520523854709
:105080006310F50218408967938777320145E3DBA7
:10509000E7FCEFF07FED2244B24041016FC01FEC0E
:1050A00017B5010013058532EFF0BFEC0945EFF0AD
:1050B000BFEB2244B24041016FC05FEA17B5010067
:1050C000130585326FF0FFEA17B50100130545326D
:1050D0006FF03FEA411122C426C206C6856417B4A8
:1050E000010013046431938784380100FD17F5FF34
:1050F0002285EFF01FE8C5BF15A9411106C6792921
:10510000054781476316E500B2403E854101828034
:1051100017B501001305852BEFF0BFE5B2408947B5
:105120003E85410182807370043001A082807370DB
:10513000043001A0797126D24AD04ECE52CC56CA44
:1051400006D622D417BA0100130A4A4797BA0100BB
:10515000938A0A46930450050549B1490145EFD0A9
:10516000DF91EFD0BFFDEFC07FE12A8403250A0065
:105170006C0081461306F00A02C697B7010023A50A
:105180009742EFB01F9709C597B7010023A02743A7
:10519000EFC0DFDE33048540130414F5EFD05FFC6D
:1051A000014563F6890097B7010023A1274197B70E
:1051B000010023AB973EEFD05F8CEFD03FF8EFC0FC
:1051C000FFDB2A8403250A0081461306F00A6C00DF
:1051D00097B7010023AA973CEFB0FFA409C597B782
:1051E000010023A5273DEFC07FD933048540130478
:1051F00014F5EFD0FFF683A70A0063F6890017B70E
:1052000001002325273B850717B70100232E973878
:1052100017B70100232EF73891B7397126DA4AD82B
:105220004ED652D456D25AD05ECE62CC66CA06DE74
:1052300022DC6AC817BA0100130A4A3817B90100FC
:105240001309893697BB0100938B0B3797BC01007C
:10525000938C4C36294C054B914A85499304500553
:1052600002C401463314CC00EFD05FEDEFC01FD174
:105270002A8D03250A00814622866C00EFB0BF9A72
:1052800009C597B7010023A33733EFC03FCF330DD4
:10529000A541EFD0FFEC9307C40063768D0017B7EC
:1052A00001002325373163F1A727224697B7010074
:1052B00023AE372F050632C4E3D6CAFA02C403254B
:1052C0000A00814601462C00EFB0BF82630A6525C3
:1052D00097B7010023AC372DA24785073EC4E3D022
:1052E000FAFE02C401463314CC00EFD03FE5EFC014
:1052F000FFC82A8D03250A00814622862C00EFB0C4
:105300004FFF09C597B7010023A2372BEFC01FC776
:10531000330DA541EFD0DFE49307C40063768D0021
:1053200017B701002324372963FAA71D224697B730
:10533000010023AD3727050632C4E3D6CAFA03A518
:105340000B0097B7010023A10726EFC03F848327F6
:105350000900638997005145EFD0AF848327090086
:10536000E39B97FE5145EFD0CF8397B7010023AD64
:10537000072202C403250A00814601466C00EFB0F3
:105380009F8A814601462C006306650197B701009C
:1053900023AE372103250A00EFB0AFF583270900BC
:1053A00095456306650117B701002321372103A541
:1053B0000B006396970097B7010023A9371FEFC032
:1053C000EFEA83270900894503A50B006396970040
:1053D00097B7010023AC371DEFC04FE9A2478507FF
:1053E0003EC4E3D9FAF88327090051456389970041
:1053F000EFC03FFB832709005145E39B97FEEFC0B9
:105400005FFA97B7010023A1071A02C403250A0017
:10541000814601466C00EFB01F81630D650F97B7A1
:10542000010023A53719A24785073EC4E3D0FAFE41
:1054300003A50B00EFC08FF5832709006389970050
:105440005145EFC01FF683270900E39B97FE5145A6
:10545000EFC03FF597B7010023A8071402C4032546
:105460000A00814601462C00EFB0AFE881460146B4
:105470006C006306650197B7010023A93713032564
:105480000A00EFB04FFA83270900954563066501CE
:1054900017B70100232C371103A50B006396970063
:1054A00097B7010023A43711EFC04FDC8327090011
:1054B000894503A50B006396970097B7010023A7C2
:1054C000370FEFC0AFDAA24785073EC4E3D9FAF839
:1054D00083270900514563899700EFC09FEC83271C
:1054E00009005145E39B97FEEFC0BFEB83A70C007B
:1054F000850717B70100232FF70A9DB3224605063B
:1055000032C4E3D2CADE25BD2246050632C4E3DB3F
:10551000CAD46DB3A24785073EC4E3D9FAEE09BFEA
:10552000A24785073EC4E3DCFAD865BB41110146BA
:105530009145154506C6EFB06F9997B50100938563
:10554000E5EC97B7010023ABA706EFB0BFE08148B9
:10555000014881470D4781461306004097B5010079
:105560009385C5EB17050000130565CBEFB0FFF67B
:10557000B2408148014897B701009387E703094784
:1055800081461306004097B501009385A5E91705EC
:105590000000130565BA41016FB03FF497B70100F1
:1055A00093870701984397B70100938767FF90435C
:1055B00097B7010093870700944397B7010093873B
:1055C00067FE9C4301456306C700B387F640333549
:1055D000F00097B70100938767FD9C4317B6010061
:1055E0002320E6FC17B70100232ED7FAFD17B337A7
:1055F000F000B307F0407D8D82800000B305B50058
:10560000930705006386B70003C70700631607000A
:105610003385A74067800000938717006FF09FFED7
:10562000130101FB23229104232C41032322910324
:10563000232611042324810423202105232E310352
:10564000232A510323286103232671032324810382
:105650002320A103232EB101930C0500138A05001A
:105660009304000063DE05003305A0403337A0003B
:10567000B305B040930C0500338AE5409304F0FF76
:1056800063DA06003306C040B337C000B306D0402B
:10569000B386F640930A06009389060013840C0033
:1056A00013090A006396062817BB0100130B8BC071
:1056B0006370CA16B70701006372F6149307F00F00
:1056C00063F4C70093098000B3573601330BFB0026
:1056D00083470B0013050002B3873701B309F54078
:1056E000638C0900B3153A01B3D7FC00B31A360135
:1056F00033E9B70033943C0113DB0A0193050B0037
:1057000013050900EF00507C130A050093050B00F8
:10571000939B0A0113050900EF00907693DB0B01C0
:105720009305050013850B00EF00D072131A0A01D0
:1057300093570401B367FA0063FAA700B3875701D0
:1057400063E6570163F4A700B38757013389A74085
:1057500093050B0013050900EF001077130A0500ED
:1057600093050B0013050900EF0090711314040159
:1057700093050500131A0A0113850B001354040145
:10578000EF00506D33648A00637AA400330454013F
:10579000636654016374A400330454013304A440C9
:1057A0003354340193050000638A040033048040BD
:1057B000B3378000B305B040B385F540130504004E
:1057C0008320C104032481048324410403290104A8
:1057D0008329C103032A8103832A4103032B010385
:1057E000832BC102032C8102832C4102032D010271
:1057F000832DC1011301010567800000B707000177
:1058000093090001E362F6EC930980016FF0DFEB8E
:10581000631A06009305000013051000EF005066A0
:10582000930A0500B707010063FAFA0E9307F00F19
:1058300063F4570193098000B3D73A01330BFB009F
:1058400083470B001305000233095A41B387370120
:10585000B309F540E38209EAB39A3A01335BFA00EF
:10586000B3153A01B3D7FC0093DB0A0133E9B70063
:1058700013050B0093850B00EF001065130A05005C
:1058800093850B00139C0A0113050B00EF00505F7A
:10589000135C0C019305050013050C00EF00905BF1
:1058A000131A0A0193570901B367FA0033943C01B4
:1058B00063FAA700B387570163E6570163F4A700B3
:1058C000B3875701338BA74093850B0013050B005B
:1058D000EF00905F130A050093850B0013050B0082
:1058E000EF00105A9305050013050C00EF009056C9
:1058F00093160901131A0A0193D60601B366DA005A
:1059000063FAA600B386560163E6560163F4A60067
:10591000B38656013389A6406FF01FDEB70700013A
:1059200093090001E3EAFAF0930980016FF0DFF0D8
:105930006376DA0093050A006FF01FE7B7070100EE
:1059400063FAF604930BF00F33B5DB001315350043
:1059500033D7A60097B701009387C795B387E700B1
:1059600083CB070093050002B38BAB00338B7541EB
:10597000631C0B0263E4460163EACC003384CC4031
:10598000B306DA4033B98C00338926419305090008
:105990006FF09FE1B707000113050001E3EAF6FA93
:1059A000130580016FF0DFFAB3966601335D76016F
:1059B000336DDD00B35D7A01B3156A0133DC7C0120
:1059C00013540D01336CBC0013850D0093050400C6
:1059D000B3196601EF00504F930A050093050400C8
:1059E00013850D0033996C01931C0D01EF00504994
:1059F00093DC0C01130A05009305050013850C00C8
:105A0000EF005045939A0A0113570C0133E7EA005F
:105A1000930D0A00637EA7003307A701930DFAFFD9
:105A20006368A7016376A700930DEAFF3307A70118
:105A3000330AA7409305040013050A00EF00D0487D
:105A400093050400930A050013050A00EF00504374
:105A5000930505001304050013850C00EF00903F2B
:105A600093150C01939A0A0193D50501B3E5BA0089
:105A70001307040063FEA500B385A5011307F4FF17
:105A800063E8A50163F6A5001307E4FFB385A5014C
:105A9000939D0D01B70C0100B3EDED001384FCFFE5
:105AA000B3F78D0033F48900338AA54013850700CE
:105AB000930504002326F10093DD0D01EF009039DA
:105AC00093050400930A050013850D00EF0090383C
:105AD00013DC090193050C002324A10013850D009C
:105AE000EF0050378327C10013040C009305040016
:105AF000130C050013850700EF00D03583268100C5
:105B000013D70A013305D5003307A7006374D70004
:105B1000330C9C01B70701009387F7FF93550701EA
:105B20003377F70013170701B3F7FA00B385850140
:105B3000B307F7006366BA00631EBA00637CF9001E
:105B400033863741B3B7C700B385A541B385F54068
:105B500093070600B307F9403339F900B305BA409B
:105B6000B385254133947501B3D767013364F400DD
:105B7000B3D565016FF05FC3130101FD23229102CC
:105B8000232A5101232611022324810223202103E9
:105B9000232E3101232C4101232861012326710189
:105BA00023248101232291012320A101930A0500CE
:105BB00093840500639E06381304060093090500CC
:105BC00017A901001309096F63F8C512B70701008F
:105BD000138B05006378F6101307F00F3337C700F7
:105BE00013173700B357E6003309F900834609005D
:105BF0003387E60093060002B386E640638C060016
:105C0000B394D40033D7EA003314D600336B970033
:105C1000B399DA00935A040193850A0013050B0027
:105C2000EF00902A1309050093850A00931B0401D5
:105C300013050B00EF00D02493DB0B019304050048
:105C40009305050013850B00EF00D02013190901FF
:105C500093D70901B367F900138A040063FEA70014
:105C6000B3878700138AF4FF63E8870063F6A70011
:105C7000138AE4FFB3878700B384A74093850A00A3
:105C800013850400EF0050241309050093850A00D2
:105C900013850400EF00D01E9399090193040500B9
:105CA000930505001319090113850B0093D9090108
:105CB000EF00501AB36939011386040063FCA90090
:105CC000B30934011386F4FF63E6890063F4A90085
:105CD0001386E4FF13140A013364C400130A00009E
:105CE0006F000013B707000113070001E36CF6EE25
:105CF000130780016FF01FEF138A0600631A060076
:105D00009305000013051000EF0090171304050021
:105D1000B7070100637EF4129307F00F63F4870066
:105D2000130A8000B35744013309F90003470900FF
:105D30009306000233074701B386E64063940612D8
:105D4000B3848440130A1000135B040193050B0015
:105D500013850400EF0050171309050093050B008D
:105D600013850400931B0401EF00901193DB0B01DA
:105D7000930405009305050013850B00EF00900DBB
:105D80001319090193D70901B367F900938A040035
:105D900063FEA700B3878700938AF4FF63E8870058
:105DA00063F6A700938AE4FFB3878700B384A74014
:105DB00093050B0013850400EF0010111309050073
:105DC00093050B0013850400EF00900B93990901D4
:105DD00093040500930505001319090113850B00B1
:105DE00093D90901EF001007B36939011386040044
:105DF00063FCA900B30934011386F4FF63E689004C
:105E000063F4A9001386E4FF13940A013364C40009
:105E10001305040093050A008320C10203248102B4
:105E200083244102032901028329C101032A81013C
:105E3000832A4101032B0101832BC100032C810024
:105E4000832C4100032D0100130101036780000032
:105E5000B7070001130A0001E366F4EC130A80019E
:105E60006FF05FEC3314D40033DAE400B399DA0056
:105E700033D7EA00935A0401B394D40093850A00FF
:105E800013050A00336B9700EF0010041309050097
:105E900093850A0013050A00931B0401EF00407E5E
:105EA00093DB0B01930405009305050013850B009C
:105EB000EF00407A1319090113570B013367E9000A
:105EC000138A0400637EA70033078700138AF4FF58
:105ED000636887006376A700138AE4FF33078700AF
:105EE000B304A74093850A0013850400EF00C07D2A
:105EF0001309050093850A0013850400EF0040781C
:105F0000930405009305050013850B00EF008074D2
:105F100013170B011357070113190901B367E900A0
:105F20001387040063FEA700B38787001387F4FF7D
:105F300063E8870063F6A7001387E4FFB387870051
:105F4000131A0A01B384A740336AEA006FF0DFDF57
:105F500063ECD51EB707010063F4F6041307F00FD6
:105F6000B335D7009395350033D7B60097A7010016
:105F700093874734B387E70003C70700130A00027B
:105F80003307B700330AEA4063160A02130410000D
:105F9000E3E096E833B6CA00134416006FF05FE7FB
:105FA000B707000193050001E3E0F6FC93058001CB
:105FB0006FF09FFBB35CE600B3964601B3ECDC00E8
:105FC00033D4E40093DB0C01B397440133D7EA00E8
:105FD00093850B0013050400336BF700B3194601DA
:105FE000EF00806E1309050093850B001305040074
:105FF000139C0C01EF00C068135C0C0193040500B6
:106000009305050013050C00EF00C0641319090186
:1060100013570B013367E90013840400637EA70064
:10602000330797011384F4FF636897016376A70031
:106030001384E4FF33079701B304A74093850B0053
:1060400013850400EF0040681309050093850B00D9
:1060500013850400EF00C06293040500930505005A
:1060600013050C00EF00005F93170B0113190901D2
:1060700093D70701B367F9001386040063FEA700F6
:10608000B38797011386F4FF63E8970163F6A700CF
:106090001386E4FFB387970113140401B70B0100C3
:1060A0003364C4001389FBFF337D240133F92901D4
:1060B000B384A7409305090013050D00EF00805934
:1060C000935C040193050900130B050013850C0074
:1060D000EF00405893D90901130C0500938509007E
:1060E00013850C00EF000057130905009385090084
:1060F00013050D00EF0000563305850193570B0182
:106100003385A7006374850133097901935705012D
:10611000B387270163E6F402E392F4BCB7070100FA
:106120009387F7FF3375F50013150501337BFB00EB
:1061300033964A0133056501130A0000E37AA6CCC1
:106140001304F4FF6FF09FB9130A0000130400005A
:106150006FF01FCC130101FB23248104232291043F
:10616000232E31032322910323261104232021050A
:10617000232C4103232A510323286103232671037F
:10618000232481032320A103232EB101930C0500B6
:10619000938905001304050093840500639E062679
:1061A00013090600138A060097AA0100938A8A1031
:1061B00063F4C514B70701006376F6129307F00F76
:1061C00063F4C700130A8000B3574601B38AFA008C
:1061D00003C70A001305000233074701330AE540ED
:1061E000630C0A00B395490133D7EC00331946011B
:1061F000B364B70033944C01935A090193850A00A4
:1062000013850400EF00404C9309050093850A00B4
:10621000131B090113850400EF008046135B0B017B
:106220009305050013050B00EF00C0429399090187
:1062300093570401B3E7F90063FAA700B387270176
:1062400063E6270163F4A700B3872701B384A7405F
:1062500093850A0013850400EF00004793090500A9
:1062600093850A0013850400EF0080411314040194
:10627000930505009399090113050B0013540401BC
:10628000EF00403D33E48900637AA4003304240125
:10629000636624016374A400330424013304A4401E
:1062A00033554401930500008320C1040324810475
:1062B00083244104032901048329C103032A8103A0
:1062C000832A4103032B0103832BC102032C810288
:1062D000832C4102032D0102832DC101130101050D
:1062E00067800000B7070001130A0001E36EF6ECB7
:1062F000130A80016FF05FED631A0600930500003A
:1063000013051000EF00C03713090500B70701009F
:10631000637AF90E9307F00F63F42701130A8000E4
:10632000B3574901B38AFA0003C70A0013050002F4
:10633000B384294133074701330AE540E30E0AEAF3
:1063400033194901B3DAE900B395490133D7EC00B9
:1063500093540901336BB70013850A009385040039
:10636000EF0080369309050093850400931B090113
:1063700013850A00EF00C03093DB0B019305050085
:1063800013850B00EF00002D9399090193570B0122
:10639000B3E7F90033944C0163FAA700B3872701F0
:1063A00063E6270163F4A700B3872701B38AA740F8
:1063B0009385040013850A00EF000031930905005E
:1063C0009385040013850A00EF00802B93050500D8
:1063D00013850B00EF00002893150B019399090119
:1063E00093D50501B3E5B90063FAA500B38525018E
:1063F00063E6250163F4A500B3852501B384A540B8
:106400006FF09FDFB7070001130A0001E36AF9F09C
:10641000130A80016FF0DFF0E3E8D5E8B707010069
:1064200063FCF604930BF00F33B5DB001315350056
:1064300033D7A60097A701009387C7E7B387E70084
:1064400083CB070093050002B38BAB00338B754100
:10645000631E0B0263E4360163EACC003384CC4054
:10646000B386D94033B58C00B384A640130504002D
:10647000938504006FF05FE3B70700011305000187
:10648000E3E8F6FA130580016FF09FFAB396660110
:10649000335D7601336DDD0033D47901B395690145
:1064A00033DC7C0193540D01336CBC0013050400F4
:1064B00093850400B31A6601EF000021130A05005A
:1064C000938504001305040033996C01931C0D019E
:1064D000EF00001B93DC0C0113040500930505007D
:1064E00013850C00EF000017131A0A0113570C0153
:1064F0003367EA00130A0400637EA7003307A7018D
:10650000130AF4FF6368A7016376A700130AE4FF88
:106510003307A701B309A740938504001385090039
:10652000EF00801A93850400130405001385090009
:10653000EF000015930505009304050013850C007A
:10654000EF00401193150C011314040193D50501BC
:10655000B365B4001387040063FEA500B385A501ED
:106560001387F4FF63E8A50163F6A5001387E4FF32
:10657000B385A501131A0A01B70C0100336AEA00BA
:106580001384FCFFB3778A0033F48A00B384A540F8
:1065900013850700930504002326F100135A0A010E
:1065A000EF00400B930905009305040013050A0052
:1065B000EF00400A13DC0A01930D050093050C005F
:1065C00013050A00EF0000098327C100130A050024
:1065D00093050C0013850700EF00C0073305B501D4
:1065E00013D709013307A7006374B701330A9A016F
:1065F000B70701009387F7FF935507013377F7003B
:1066000013170701B3F7F900B3854501B307F70086
:1066100063E6B400639EB400637CF900338657419F
:10662000B3B7C700B385A541B385F540930706000E
:10663000B307F9403339F900B385B440B385254138
:1066400033947501B3D767013365F400B3D56501A1
:106650006FF09FC5130605001305000093F61500A3
:10666000638406003305C50093D515001316160084
:10667000E39605FE678000006340050663C60506D5
:1066800013860500930505001305F0FF630C060251
:1066900093061000637AB6006358C0001316160004
:1066A00093961600E36AB6FE1305000063E6C50084
:1066B000B385C5403365D50093D616001356160032
:1066C000E39606FE6780000093820000EFF05FFB18
:1066D00013850500678002003305A04063D80500DC
:1066E000B305B0406FF0DFF9B305B040938200000E
:1066F000EFF01FF93305A04067800200938200008D
:1067000063CA0500634C0500EFF09FF71385050091
:1067100067800200B305B040E35805FE3305A04092
:10672000EFF01FF63305B0406780020097A7010025
:106730009387C7E3944317A701001307E7E11843C2
:10674000C8C2637BE50017A701001307A7E1084350
:106750008C4391056F90DFDE411122C406C617A756
:106760000100130767E02A8408438C439105EF90EA
:106770003FDD97A70100938767DC9C436376F400B5
:1067800097A7010023AC87DAB240224441018280FE
:1067900097A70100938787DD984394437C43FD17B7
:1067A0007CC3FC4299E3736004308280011122CCE7
:1067B00026CA2A84AE844AC84EC652C456C206CEE1
:1067C000EFB0CFFA1C4003290401B7090001B3E57B
:1067D0009700930AC4000CC08144FD19370A0002D7
:1067E0001840638C2A03032609004A85B3654701D4
:1067F000B376360193175600758F0329490063C499
:10680000070001E7F1BFE39DE6FC9317760063D331
:106810000700D58CEFC0EFE4E1B793C4F4FFF98C27
:1068200004C0EFB0BF990840F2406244D2444249EC
:10683000B249224A924A05618280411106C622C4A9
:10684000EFE0DFCE17E7FFFF1307477E81460546DF
:106850009305400617A50100130585BAEFD06FB464
:1068600019C92A84EFB08FF12A86014781468545F0
:106870002285EFD0AFBFEFB0EFC9B240224401454F
:0468800041018280D0
:02000004800278
:100000002C47FEFF2A48FEFF3447FEFF2A48FEFF2A
:100010002A48FEFF2A48FEFF2A48FEFF4C47FEFF03
:100020002A48FEFF2A48FEFF6647FEFF7247FEFF92
:100030002A48FEFF8447FEFF9047FEFF9047FEFFE1
:100040009047FEFF9047FEFF9047FEFF9047FEFF60
:100050009047FEFF9047FEFF9047FEFF2A48FEFFB5
:100060002A48FEFF2A48FEFF2A48FEFF2A48FEFFD4
:100070002A48FEFF2A48FEFF2A48FEFF2A48FEFFC4
:100080002A48FEFF2A48FEFF2A48FEFF2A48FEFFB4
:100090002A48FEFF2A48FEFF2A48FEFF2A48FEFFA4
:1000A0002A48FEFF2A48FEFF2A48FEFF2A48FEFF94
:1000B0002A48FEFF2A48FEFF2A48FEFF2A48FEFF84
:1000C0002A48FEFF2A48FEFF2A48FEFF2A48FEFF74
:1000D0002A48FEFF2A48FEFF2A48FEFF2A48FEFF64
:1000E0002A48FEFF2A48FEFF2A48FEFF2A48FEFF54
:1000F0002A48FEFF2A48FEFF2A48FEFF2A48FEFF44
:10010000C447FEFFDA47FEFF2A48FEFF2A48FEFFEB
:100110002A48FEFF2A48FEFF2A48FEFF2A48FEFF23
:100120002A48FEFF2048FEFF2A48FEFF2A48FEFF1D
:10013000D245FEFF8A46FEFF2A48FEFF2A48FEFF00
:10014000C046FEFF2A48FEFF1847FEFF2A48FEFF72
:100150002A48FEFF4647FEFF384BFEFF8C4BFEFF52
:10016000404BFEFF8C4BFEFF8C4BFEFF8C4BFEFF8B
:100170008C4BFEFF324AFEFF8C4BFEFF8C4BFEFF8A
:100180004C4AFEFF584AFEFF8C4BFEFF6A4AFEFFB8
:10019000764AFEFF764AFEFF764AFEFF764AFEFF6B
:1001A000764AFEFF764AFEFF764AFEFF764AFEFF5B
:1001B000764AFEFF8C4BFEFF8C4BFEFF8C4BFEFF06
:1001C0008C4BFEFF8C4BFEFF8C4BFEFF8C4BFEFFDF
:1001D0008C4BFEFF8C4BFEFF8C4BFEFF8C4BFEFFCF
:1001E0008C4BFEFF8C4BFEFF8C4BFEFF8C4BFEFFBF
:1001F0008C4BFEFF8C4BFEFF8C4BFEFF8C4BFEFFAF
:100200008C4BFEFF8C4BFEFF8C4BFEFF8C4BFEFF9E
:100210008C4BFEFF8C4BFEFF8C4BFEFF8C4BFEFF8E
:100220008C4BFEFF8C4BFEFF8C4BFEFF8C4BFEFF7E
:100230008C4BFEFF8C4BFEFF8C4BFEFF8C4BFEFF6E
:100240008C4BFEFF8C4BFEFF8C4BFEFF8C4BFEFF5E
:100250008C4BFEFF8C4BFEFFAA4AFEFFD84AFEFFE6
:100260008C4BFEFF8C4BFEFF8C4BFEFF8C4BFEFF3E
:100270008C4BFEFF8C4BFEFF8C4BFEFF2E4BFEFF8C
:100280008C4BFEFF8C4BFEFF9048FEFF8A49FEFF21
:100290008C4BFEFF8C4BFEFFFC49FEFF8C4BFEFFA0
:1002A000224AFEFF8C4BFEFF8C4BFEFF864BFEFF6F
:1002B000000102020303030304040404040404040D
:1002C00005050505050505050505050505050505DE
:1002D00006060606060606060606060606060606BE
:1002E00006060606060606060606060606060606AE
:1002F000070707070707070707070707070707078E
:10030000070707070707070707070707070707077D
:10031000070707070707070707070707070707076D
:10032000070707070707070707070707070707075D
:10033000080808080808080808080808080808083D
:10034000080808080808080808080808080808082D
:10035000080808080808080808080808080808081D
:10036000080808080808080808080808080808080D
:1003700008080808080808080808080808080808FD
:1003800008080808080808080808080808080808ED
:1003900008080808080808080808080808080808DD
:1003A00008080808080808080808080808080808CD
:1003B000546D725100000000546D7220537663003A
:1003C000286E756C6C2900004572726F7220696E20
:1003D00020416C74426C6F636B207461736B73208B
:1003E0000D0A00006D69616F750A00006D69616F2B
:1003F00075320A0068756E6772790A004368656332
:100400006B54696D65720000416C74426C6F636B74
:10041000517565756500000046425465737431007E
:0804200046425465737432007A
:100428001000000000000000017A5200017C010168
:100438001B0D02005000000018000000DC51FEFFF8
:100448005805000000440E507489039406990B81E6
:1004580001880292049305950796089709980A9AC5
:100468000C9B0D036C010AC144C844C944D244D34F
:1004780044D444D544D644D744D844D944DA44DB98
:10048800440E00440B0000004C0000006C0000000B
:10049800E056FEFFDC05000000440E30708903952D
:1004A8000781018802920493059406960897099893
:1004B8000A990B9A0C0370020AC144C844C944D271
:1004C80044D344D444D544D644D744D844D944DA50
:1004D800440E00440B00000050000000BC00000067
:1004E8006C5CFEFF0005000000440E507488028911
:1004F800039305990B810192049406950796089732
:1005080009980A9A0C9B0D0320010AC144C844C9E2
:1005180044D244D344D444D544D644D744D844D907
:0C05280044DA44DB440E00440B000000E9
:0805BC00FC8F010009000000A2
:040000058000004037
:00000001FF
